S01B00006F70656E626C745F656B5F6C6D3373363936352E737265632E
S113000008020020DD7C0000217D0000217D00002D
S1130010217D0000217D0000217D0000217D000064
S1130020217D0000217D0000217D0000217D000054
S1130030217D0000217D0000217D0000217D000044
S1130040217D0000217D0000217D0000217D000034
S1130050217D0000217D0000217D0000217D000024
S1130060217D0000217D0000217D0000217D000014
S1130070217D0000217D0000217D0000217D000004
S1130080217D0000217D0000217D0000217D0000F4
S1130090217D0000217D0000217D0000217D0000E4
S11300A0217D0000217D0000217D0000217D0000D4
S11300B0217D0000217D0000217D0000217D0000C4
S11300C0217D0000217D0000217D0000217D0000B4
S11300D0217D0000217D0000217D0000217D0000A4
S11300E0217D0000217D0000217D0000217D000094
S11300F003E00B780370491C401C13005A1E002BAC
S1130100F7D1704701E00170401C13005A1E002B08
S1130110F9D1704710B400231400621E002C06D0DD
S113012003780C781B1B491C401C002BF4D01800CE
S113013010BC704700E0401C0278002A02D002780C
S11301408A42F8D10078704770B5040020790028FD
S113015023D0256B01232A0014F13401607802F0C6
S113016088F9002801D0012018E000202071606A7D
S1130170854212D3606AE169081885420DD2E67897
S113018009E0E069451901232A0014F1340160787B
S113019002F06FF9761E022EF3D2002070BD38B53E
S11301A004000D00206B854212D02000FFF7CCFF25
S11301B0002801D001200CE001232A0014F13401AD
S11301C0607802F009F9002801D0012001E02563DC
S11301D0002032BD38B504002000FFF7B5FF05004C
S11301E0EDB2002D5DD12078032852D1607900282A
S11301F04FD0002020634FF40072002114F134002A
S1130200FFF780FF552084F83202AA2084F83302D5
S1130210522084F83400522084F83500612084F898
S11302203600412084F83700722084F818027220C6
S113023084F81902412084F81A02612084F81B0210
S1130240206984F81C02206980B2000A84F81D0227
S11302502069000C84F81E022069000E84F81F0235
S1130260E06884F82002E06880B2000A84F8210281
S1130270E068000C84F82202E068000E84F823028F
S11302800123626914F13401607802F0F2F800206D
S1130290607100220021607802F049F9002800D042
S11302A001252800C0B232BD891E8269921E914286
S11302B001D3002003E08278C06A02FB010070478A
S11302C0F8B504000D00022D02D3A069854201D3C4
S11302D0012014E02078012804D00ED303283ED056
S11302E02AD30AE02F0017EB5707606A10EB572157
S11302F02000FFF754FF002802D05FF0FF30F2BD6A
S1130300F805C00D204490F834607F1C606A10EB3F
S113031057212000FFF743FF0028EED1F805C00D58
S1130320204490F8340056EA0026E80701D5300945
S113033001E03005000DE2E7606A10EB15212000B2
S1130340FFF72DFF0028D8D16800C005C00D204458
S113035034304178007850EA012080B2CFE7606AF7
S113036010EBD5112000FFF71AFF0028C5D1A80013
S1130370C005C00D20443430C1788278120452EA9A
S11303800161427851EA02210078084320F070406C
S1130390B5E7F8B504000D001600022D02D3A069DC
S11303A0854201D3022072E02078012804D06BD367
S11303B003284CD038D367E02F0017EB5707606A47
S11303C010EB57212000FFF7EAFEC0B200285CD1F1
S11303D0F805C00D204410F13401E80705D508786C
S11303E010F00F0050EA061000E0300008707F1C87
S11303F001202071606A10EB57212000FFF7CFFE27
S1130400C0B2002841D1F905C90D21443431EA07AD
S113041001D5320906E00A7812F0F002330A13F02B
S11304200F031A430A7030E0606A10EB15212000B4
S1130430FFF7B5FEC0B2002827D16900C905C90D70
S1130440214434310E70B6B2320A4A701DE0606A3B
S113045010EBD5112000FFF7A2FEC0B2002814D182
S1130460A900C905C90D21443431CA78120612F015
S1130470704216430E70320092B2120A4A70320C65
S11304808A70320ECA7000E0022001212171C0B2CC
S1130490F2BDF8B504000E00022E02D3A069864214
S11304A001D3022527E0002509E0206910F1010F9E
S11304B004D02069401C2061012060713E00A069C5
S11304C0864218D231002000FFF7FAFE0700002F01
S11304D011D0012F01D102250DE017F1010F01D137
S11304E0012508E0002231002000FFF752FF05003B
S11304F0EDB2002DD9D02800C0B2F2BDF8B5040089
S11305000E00002E07D1E768002F02D0A0698742B1
S11305100DD301270BE031002000FFF7D1FE0228A4
S113052001D2012043E0A169884240D337003D0055
S11305306D1CA069854204D30225AF4201D200207C
S113054035E029002000FFF7BBFE00281DD17FF015
S1130550704229002000FFF71CFFC0B2002806D11A
S1130560002E04D02A0031002000FFF712FFC0B291
S1130570002814D1E560206910F1010F16D020691C
S1130580401E20610120607110E010F1010F01D0C4
S1130590012800D10BE0BD42CAD1002007E0C0B25F
S11305A0012802D15FF0FF3500E001252800F2BDEB
S11305B070B504000D00E580A068012803D021680F
S11305C08969884201D3022048E0002805D12168C6
S11305D00978032901D12068806A00280FD1E060DE
S11305E028002168098980B2884201D3022035E0BD
S11305F02068806AADB210EB1510206125E02168F7
S1130600897889B20E0100E0AD1B2900320089B25D
S113061092B2914210D301002068FFF751FE10F10D
S1130620010F01D1012019E0022803D3216889694F
S11306308842E9D3022011E0E06001002068FFF75E
S113064033FEADB210EB151020612068ADB215F089
S11306500F014901084434306061002070BDF8B5D1
S113066004000D00E088461CB6B2002E02D02069BA
S1130670002801D1042081E00F20064274D12069B2
S1130680401C2061E068002807D1300021680989F6
S113069080B2884268D3042070E0B6B220688078C3
S11306A0401E10EA161F5FD1E1682068FFF708FEBC
S11306B00700022F01D2022060E017F1010F01D1DF
S11306C001205BE020688069874247D3002D01D177
S11306D0042053E0E1682068FFF710FF0700002FB3
S11306E001D107204AE0012F01D1022046E017F191
S11306F0010F01D1012041E02068FFF725FD00280A
S113070001D001203AE04FF4007200212068343017
S1130710FFF7F8FC39002068FFF7C6FD216808637D
S1130720002505E02068006B401C216808636D1CEF
S1130730280021688978C0B2884209D20120216842
S113074008712068FFF700FD0028EBD0012015E0B8
S11307502068006BEDB2401B21680863E760390034
S11307602068FFF7A1FD2061E6802068B6B216F08C
S11307700F0149010844343060610020F2BD70B5B6
S113078004000D0000212000FFF712FFC0B2002872
S11307901BD1002621692068FFF701FDC0B20028A3
S11307A013D161690978E52903D0616909780029C1
S11307B003D1761CAE4201D107E0002601212000BE
S11307C0FFF74DFFC0B20028E4D0C0B270BDCA7EAE
S11307D08B7E53EA022292B20078032806D1487D28
S11307E0097D51EA002080B252EA004210007047AD
S11307F081760A0092B2120AC2760A0C0275090CBA
S113080089B2090A417570472DE9F04104000D00D1
S1130810287830F04000401E0D2101FB00F600272F
S11308205FF00108DFF82C0DC05D28444078DFF844
S1130830241DC95D695C51EA00201FFA88F8B8F1EB
S1130840000F11D080B201F0D8FF8046FF2E09D2EC
S113085034F8160001F0D1FF761C414689B280B20B
S1130860814208D0002018E080B24FF6FF71884220
S113087001D0002011E07F1C0D2FD3D3287840062F
S11308800AD51FFA88F8B8F1000F05D034F816001D
S1130890002801D0002000E00120BDE8F08170B400
S11308A00A7812F03F02521E0D235A4300230124FA
S11308B0DFF8A05CED5C0D446D78DFF8986CF65CB5
S11308C08E5D56EA0525A4B2002C11D0FF2A01D36F
S11308D0002018E02C0020F81240521C5B1C0D2B49
S11308E0E6D3097849060DD5FF2A08D300200AE08B
S11308F0ADB24FF6FF76B542F0D0002003E0002100
S113090020F81210012070BC7047F0B44B730F2311
S1130910CB7200230B7300238B760023CB76D2B2E9
S1130920531E0D2404FB03F40025ADB22E00ADB21A
S11309304FF6FF739D4202D030F81450641CDFF868
S1130940143C9B5DCD542B009BB21B0ADFF8047C46
S1130950BF5D0F447B70ADB2002D01D14FF6FF7522
S1130960761C0D2EE3D3ADB24FF6FF739D4203D038
S113097030F81400002801D152F040020A70F0BC93
S113098070477CB5040016001D000B222000FFF701
S1130990AFFBADB2062D0ADB280080B2E90311EBF0
S11309A0500031880D18B61C30880028F4D1072077
S11309B0ADB2102195FBF1F201FB12513031C9B2F5
S11309C03A2900DBC91D6A461154401EADB21021FC
S11309D095FBF1F5ADB2002DEAD17E216A461154A2
S11309E0002100E0491C814202D2625C202AF9D134
S11309F00A00511C082803D26B461B5C401C00E013
S1130A002023A3540829F3D373BD00210B220B0028
S1130A10DBB2C90111EB530103785918401C521E73
S1130A20002AF4D10800C0B270472DE9F041050056
S1130A3000212800FFF7BCFD0400E4B2002C02D022
S1130A402000C0B227E04FF0FF0847462969286814
S1130A50FFF7A5FB0400E4B2002C1AD16E693078CC
S1130A60C0B2002801D1042413E0F17A11F03F014F
S1130A70C0B2E52804D00A070FD5C9B20F290CD09B
S1130A80FF2700212800FFF7EAFD0400E4B2002C50
S1130A90DCD02000C0B2BDE8F081C9B20F291FD15B
S1130AA0E9690029EDD0410606D596F80D8010F0CD
S1130AB0BF000700E98829843900C0B2C9B288425E
S1130AC00CD14046717BC0B2884207D13100E8693D
S1130AD0FFF79AFE002801D07F1ED2E7FF27D0E758
S1130AE0FFB2002F06D147463000FFF78EFFFFB25A
S1130AF08742CED0FF274FF6FF702884A869C07ABA
S1130B00C007BED40B22A9693000FFF703FB0028FD
S1130B10B7D1BEE72DE9F04104000D00FF26FF2701
S1130B205FF00408206900282ED021692068FFF7AF
S1130B3036FB80465FFA88F8B8F1000F24D160696B
S1130B400278D2B2002A02D15FF004081CE0C17A14
S1130B5011F03F01D2B2E52A0BD0D2B22E2A08D02E
S1130B60C9B2082901D1012300E00023DBB2AB4262
S1130B7015D0FF2600212000FFF771FD80465FFAA3
S1130B8088F8B8F1000FCDD05FFA88F8B8F1000FFB
S1130B9001D0002020614046C0B2BDE8F081C9B256
S1130BA00F291BD1510605D5477B12F0BF02160051
S1130BB0E18821843100D2B2C9B28A420CD1390011
S1130BC0427BC9B2914207D10100E069FFF767FE99
S1130BD0002801D0761ECDE7FF26CBE7F6B2002E23
S1130BE004D1FFF712FFFFB2874202D04FF6FF7025
S1130BF02084C9E72DE9F04184B00400A669E769BF
S1130C000C2231006846FFF773FA9DF80B00C00709
S1130C102CD50020F0720020E0615FF0010801E0B3
S1130C2018F101081FFA88F8B8F1640F0DDA434689
S1130C309BB23A0069463000FFF7A3FE2000FFF79D
S1130C40F4FE0500EDB2002DEAD01FFA88F8B8F1E1
S1130C50640F01D107207BE0EDB2042D02D02800FF
S1130C60C0B275E09DF80B00F072E7619DF80B00CF
S1130C70800712D55FF0000801E018F101081FFA9F
S1130C8088F837F818000028F7D11FFA88F818F107
S1130C9019000D2190FBF1F600E00126B6B23100F7
S1130CA02000FFF76CFD0500EDB2002D30D1761E5B
S1130CB0B6B2002E2CD0E088811B89B22000FFF749
S1130CC077FC0500EDB2002D22D1A069FFF79DFE4F
S1130CD0070021692068FFF762FA0500EDB2002DD4
S1130CE016D13B00DBB23200D2B26169E069FFF792
S1130CF00CFE01202168087100212000FFF7AFFCE1
S1130D000500EDB2002D03D1761EB6B2002EE0D15F
S1130D10EDB2002D1AD121692068FFF740FA0500D1
S1130D20EDB2002D12D1202200216069FFF7EAF90B
S1130D300B22A1696069FFF7DBF9A069C07A10F0A2
S1130D401800616908730120216808712800C0B285
S1130D5004B0BDE8F08138B50400E588208C4FF676
S1130D60FF71884201D1290000E0218C89B2200062
S1130D70FFF71EFCC0B200281CD121692068FFF7D0
S1130D800EFAC0B2002811D1E52162691170012167
S1130D9022681171E1882A0092B2914206D20021A0
S1130DA02000FFF75CFCC0B20028E6D0C0B20428E3
S1130DB000D10220C0B232BD2DE9F84F04008846AC
S1130DC00020D8F8009001E019F1010999F8000019
S1130DD02F28F9D099F800005C28F5D0E06900903C
S1130DE00026350003E0009820F81670761C19F8E8
S1130DF005706D1CBFB2202F05DBBFB22F2F02D0B0
S1130E00BFB25C2F09D109EB0500C8F80000BFB2DE
S1130E10202F20DA5FF0040821E0FF2E01D3062002
S1130E2093E007F0FF070121380080B201F0BCFC19
S1130E300700BFB2002F01D1062086E0BFB2802F89
S1130E40D1DABFB23900DFF8F808FFF773F90028E8
S1130E50C9D0062079E05FF0000800E0761E002E7D
S1130E600AD0009800EB460030F8027CBFB2202F75
S1130E70F4D0BFB22E2FF1D0002E01D1062064E0B1
S1130E800020009921F816000B222021A069FFF709
S1130E9039F9002500E06D1C009830F81500202871
S1130EA0F9D0009830F815002E28F4D0002D03D086
S1130EB058F0030800E0761E002E06D0009800EBE0
S1130EC0460030F8020C2E28F5D15FF00009CA461E
S1130ED05FF0080B01E058F00308009830F8157033
S1130EE06D1CBFB2002F32D1A0690078E52802D171
S1130EF00520A1690870BBF1080F01D15FEA8A0AD5
S1130F005FFA8AFA1AF00C000C2805D05FFA8AFA04
S1130F101AF00300032801D158F002085FEA887030
S1130F200FD45FFA8AFA1AF00300012801D158F0AD
S1130F3010085FFA8AFA1AF00C00042801D158F05C
S1130F400808A06980F80B800020BDE8F28FBFB2CA
S1130F50202FC0D0BFB22E2F01D1B542BBD1D9456D
S1130F6001D2B54213D1BBF10B0F02D158F00308E3
S1130F70BAE7B54201D058F00308AE42B4D3350005
S1130F805FF008095FF00B0B5FEA8A0AA5E7BFB2BE
S1130F90802F10DB0021380080B201F005FC07002F
S1130FA0BFB2002F05D0DFF89C07BFB2384410F859
S1130FB0807C58F00208BFB2002F07D0BFB23900BE
S1130FC0DFF88407FFF7B6F8002803D05F2758F04E
S1130FD003080FE0BFB2B7F141001A2802D25AF059
S1130FE0020A07E0BFB2B7F161001A2802D25AF030
S1130FF0010A203FA06900F8097019F101096CE7A2
S1131000F8B50C0014F109010269002A48D04269BC
S1131010137B00250EE0F6B2052E00D1E5261F074E
S113102005D5F6B2B6F141071A2F00D220360E705C
S1131030491C6D1C082D03D2565DF6B2202EEAD150
S1131040157A202D15D02E250D70491C08250AE08F
S1131050DF0605D5F6B2B6F141071A2F00D22036C5
S11310600E70491C6D1C0B2D03D2565DF6B2202E5A
S1131070EED1D37A2372D37F957F2D0455EA03638F
S1131080557F53EA0523157F2B432360537E157E3A
S113109055EA0323A380D37D927D52EA0322E280A2
S11310A000220A70A169002926D0E169002923D011
S11310B0A6690025016900291CD0018C4FF6FF7236
S11310C0914217D0C76901E070556D1C3888BF1C68
S11310D0010089B200290DD0002180B201F064FB27
S11310E080B2002801D1002504E0E169491E8D4247
S11310F0EAD3002500207055F1BD13B50400019812
S113110000782F2803D0019800785C2802D1019838
S1131110401C01900020A0600198007820280AD289
S113112000212000FFF744FA0021616120E02068DB
S1131130FFF74DFBA06001A92000FFF73DFEC0B200
S1131140002815D12000FFF770FCA169C97AC0B24C
S1131150002806D0C0B204280AD1490700D40520CB
S113116006E0490704D46169C87AC006DFD40520C3
S1131170C0B216BD10B5040001230A0014F13401F5
S1131180607801F029F9002801D003202DE094F8BB
S1131190330294F8321251EA002080B24AF6552103
S11311A0884201D0022020E094F86C0094F86B107F
S11311B0090251EA004094F86A100843DFF8201C41
S11311C0884201D1002010E094F8880094F8871038
S11311D0090251EA004094F886100843DFF8001C25
S11311E0884201D1002000E0012010BDF8B51500AF
S11311F002681378B3F130060A2E05D253783A2BDD
S113120002D1921C026000E0002600200860002E3B
S113121001D00B209DE1DFF8CC0B50F82640002CC8
S113122001D10C2095E10C60207800280DD0607865
S113123001F0C9F8C10708D4EDB2002D03D040076E
S113124001D50A2085E1002083E10020207066702A
S1131250607801F015F8C10701D5032079E1EDB2FA
S1131260002D03D0400701D50A2072E10025290092
S11312702000FFF77FFF0600F6B2012E1DD10020EB
S1131280C0B2002800D0401EC0B2000120444FF478
S1131290F9710844017900290FD0C17A827A1204C5
S11312A052EA0161427A51EA0221007A50EA0105C8
S11312B029002000FFF75EFF0600F6B2032E01D1DD
S11312C0012046E1F6B2002E01D00D2041E194F850
S11312D0400094F83F1051EA002080B2B0F5007F3E
S11312E001D00D2035E194F84B0094F84A1051EAEE
S11312F0002080B200280DD194F85B0094F85A10B5
S1131300090451EA006094F8591050EA012094F855
S113131058100843E06194F84410E170C9B20129FF
S113132004D0C9B2022901D00D2012E1C9B2484348
S113133094F84110A170C9B2002903D04A1EC9B261
S1131340114201D00D2004E194F8461094F8452090
S113135052EA01212181217A0F22114201D00D206C
S1131360F7E094F8481094F8472052EA012292B228
S1131370002A0DD194F8571094F85620120452EA1A
S1131380016194F8552051EA022194F854200A434B
S113139094F8431094F8423053EA012189B20029A9
S11313A001D10D20D5E089B24318268913EB161319
S11313B09A4201D20D20CCE0D21AA678B2FBF6F202
S11313C0002A01D10D20C4E0012640F6F677BA4286
S11313D000D302264FF6F677BA4200D30326921CB6
S11313E0A261256289B2491961625919E162F6B2B2
S11313F0032E16D12089002801D00D20A9E094F8ED
S1131400630094F86210090451EA006094F86110D2
S113141050EA012094F860100843A062A06980009B
S113142015E02189002901D10D2092E0616A40185C
S1131430A062F6B2022E02D1A069400007E0A069C2
S113144003214843217E11F0010111EB5000E169B1
S113145000F2FF10B1EB502F01D20D2079E05FF0C4
S1131460FF3020610020E060F6B2032E60D100203E
S1131470607194F8650094F8641051EA002080B219
S1131480401960610123626914F13401607800F04D
S1131490A3FF00284CD194F8330294F8321251EA95
S11314A0002080B24AF65521884241D194F8370091
S11314B094F83610090451EA006094F8351050EAA3
S11314C0012094F834100843DFF8EC1988422FD136
S11314D094F81B0294F81A12090451EA006094F873
S11314E0191250EA012094F818120843DFF8CC19B5
S11314F088421DD194F8230294F82212090451EA77
S1131500006094F8211250EA012094F82012084354
S1131510E06094F81F0294F81E12090451EA006076
S113152094F81D1250EA012094F81C12084320611B
S11315302670DFF88C090088401CDFF884190880C5
S1131540DFF87C090088E0800020206300202071FF
S11315500020F2BDF07C000080B500280BD00168AB
S1131560002908D001680978002904D00168C988D5
S11315708288914201D0092008E00068407800F098
S113158022FFC00701D5032000E0002002BDC0B245
S1131590002801D00B2012E0DFF84828C0B252F82E
S11315A02020002A01D000231370002901D000223A
S11315B00A70DFF83028C0B242F8201000207047CB
S11315C02DE9F2438CB004001500002C01D1092050
S11315D0B3E00020206015F01F0515F0FE026946F7
S11315E00CA8FFF703FE0600F6B2002E40F0A3801D
S11315F009A80690DFF8CC0807900C996846FFF715
S11316007CFD0600059FF6B2002E02D1002F00D10A
S113161006261C20054258D0F6B2002E0AD0F6B297
S1131620042E03D16846FFF7E5FA060055F00805D5
S1131630059F08E0F87A1121084201D0072602E04C
S1131640680700D50826F6B2002E4CD128074AD5E3
S113165001F092F8804687F80E80404680B2000A76
S1131660F8735FEA184038745FEA186078740020F1
S1131670F87200203877002078770020B8770020AF
S1131680F87739000098FFF7A2F881460021380066
S1131690FFF7AEF8012000990871B9F1000F22D0CC
S11316A00098D0F8308049460098FEF7F2FE060014
S11316B0F6B2002E17D1B9F101000099C860414675
S11316C00098FEF76CFD06000DE0F6B2002E0AD17C
S11316D0F87AC00601D5042605E0A80703D5F87AF0
S11316E0C00700D50726F6B2002E07D1280701D57A
S11316F055F020050098006BE0612762F6B2002ED9
S113170019D1A57139000098FFF761F82061F87FBD
S1131710B97F090451EA0060797F50EA0120397FDA
S11317200843E0600020A0600020A06100982060D1
S11317300098C088A0803000C0B20DB0BDE8F0832E
S1131740307D0000A87500006C7D00002DE9F04795
S1131750050016001F000C00002038602800FFF769
S1131760FBFEC0B2002801D0C0B2D8E0A8790006C0
S113177001D50220D3E0A879C00701D40720CEE028
S1131780E868A968401AB04220D206001EE0C5F8F5
S11317901890A868C005C00DD0F50078464500D261
S11317A0B0464246A868C005C00D284410F1240183
S11317B02000FEF79DFC4444A86818EB0000A860D4
S11317C0386818EB00003860B6EB0806002E00F00D
S11317D0A580A868C005DCD1A868400A2968897872
S11317E0491E11EA00085FFA88F8B8F1000F1AD10F
S11317F0A868002801D1286903E069692868FEF710
S11318005FFD022805D2A87950F08000A87102205B
S113181085E010F1010F05D1A87950F08000A8717E
S113182001207CE0686169692868FEF73DFD814616
S1131830B9F1000F05D1A87950F08000A8710220F9
S11318406DE05FFA88F818EB09095FEA562ABAF1E5
S1131850000F37D0286880785FFA88F81AEB0801FF
S1131860884205D2286880785FFA88F8B0EB080AC5
S11318705346DBB24A4621002868407800F0ACFDAC
S1131880002805D0A87950F08000A871012046E016
S1131890A879400611D5A869B0EB090050450CD2CF
S11318A04FF4007215F12401A869B0EB09004FF45C
S11318B0007358432044FEF71BFC4FF4007000FBF8
S11318C00AF878E7A86948453FF461AFA87940066B
S11318D013D50123AA6915F124012868407800F082
S11318E0C8FD002805D0A87950F08000A871012017
S11318F015E0A87910F0BF00A87101234A4615F13C
S113190024012868407800F067FD00283FF43FAFC9
S1131910A87950F08000A871012000E00020BDE803
S1131920F0872DE9F047050016001F000C00002089
S113193038602800FFF710FEC0B2002801D0C0B202
S113194060E0A879000601D502205BE0A879800751
S113195001D4072056E0E8683018E968884223D2A9
S1131960002621E0C5F81890A868C005C00DD0F580
S11319700078464500D2B04642462100A868C0051A
S1131980C00D28442430FEF7B3FBA87950F0400082
S1131990A8714444A86818EB0000A860386818EBE4
S11319A000003860B6EB0806002E20D0A868C005F9
S11319B0DAD1A868400A29688978491E11EA000822
S11319C05FFA88F8B8F1000F30D1A868002808D170
S11319D02869002809D100212868FEF78FFD2861B5
S11319E003E069692868FEF789FD00280CD1E868DE
S11319F0A968884201D2A868E860A87950F020005C
S1131A00A8710020BDE8F087012805D1A87950F01D
S1131A108000A8710220F5E710F1010F05D1A87923
S1131A2050F08000A8710120ECE76861A8794006B5
S1131A3013D50123AA6915F124012868407800F020
S1131A4018FD002805D0A87950F08000A871012065
S1131A50D8E7A87910F0BF00A87169692868FEF773
S1131A6023FC8146B9F1000F05D1A87950F080001C
S1131A70A8710220C6E75FFA88F818EB09095FEA43
S1131A80562ABAF1000F39D0286880785FFA88F8AE
S1131A901AEB0801884205D2286880785FFA88F832
S1131AA0B0EB080A5346DBB24A4621002868407866
S1131AB000F0DFFC002805D0A87950F08000A87160
S1131AC001209FE7A869B0EB0900504511D24FF4FB
S1131AD00072A869B0EB09004FF40071484304EBAD
S1131AE0000115F12400FEF703FBA87910F0BF00F4
S1131AF0A8714FF4007000FB0AF84AE7A86948454A
S1131B003FF430AFA868E9688842BFF42BAF0123E3
S1131B104A4615F124012868407800F05DFC00284D
S1131B203FF420AFA87950F08000A871012069E744
S1131B3038B504002000FFF70FFDC0B200284AD1D9
S1131B40A179890647D5A07940060FD50123A2695A
S1131B5014F124012068407800F08BFC002801D0A7
S1131B60012039E0A07910F0BF00A071E16920687C
S1131B70FEF715FBC0B200282DD1256AE87A50F093
S1131B802000E872E0682877E06880B2000A68778D
S1131B90E068000CA877E068000EE8772169280067
S1131BA0FEF726FE00F0E8FDA875010089B2090AD7
S1131BB0E975010C2976000E68760020A8740020CF
S1131BC0E874A07910F0DF00A07101202168087189
S1131BD02068FEF7FFFAC0B232BD10B50400200041
S1131BE0FFF7A6FFC0B2002801D100212160C0B2D6
S1131BF010BD2DE9F04104000D002000FFF7ACFCFE
S1131C000600F6B2002E02D03000C0B2C0E0A079C7
S1131C10000601D50220BBE0E068A84203D2A07907
S1131C20800700D4E568A0680027A760002D75D060
S1131C30216889784FF4007202FB01F8002810D063
S1131C40411EB1FBF8F16A1EB2FBF8F28A4208D3D6
S1131C50401EB8F101018843A060A0682D1A606994
S1131C6019E02069002815D100212068FEF746FC00
S1131C70012805D1A07950F08000A071022087E0EE
S1131C8010F1010F05D1A07950F08000A07101205E
S1131C907EE020616061002807D13FE06061A168B7
S1131CA018EB0101A160B5EB0805A84509D2A1799B
S1131CB0890718D501002068FEF720FC002816D1FA
S1131CC04546A1686918A160E90527D0010020688C
S1131CD0FEF7EAFA0700002F1ED1A07950F0800029
S1131CE0A071022054E001002068FEF7E9FA10F127
S1131CF0010F05D1A07950F08000A071012047E0C8
S1131D00022803D3216889698842C7D3A07950F097
S1131D108000A07102203BE017EB5527A068C005A6
S1131D202AD0A069874227D0A079400613D5012381
S1131D30A26914F124012068407800F09AFB00287D
S1131D4005D0A07950F08000A071012020E0A07996
S1131D5010F0BF00A07101233A0014F1240120689F
S1131D60407800F039FB002805D0A07950F08000BD
S1131D70A07101200CE0A761E068A168884205D247
S1131D80A068E060A07950F02000A0713000C0B2DB
S1131D90BDE8F08131B58CB00C00002203A90CA879
S1131DA0FFF724FA0500EDB2002D15D1684609901D
S1131DB0DFF810010A900C9903A8FFF79EF90500BB
S1131DC0EDB2002D08D10898002804D0210003A802
S1131DD0FFF716F900E006252800C0B20DB030BDAB
S1131DE0464154004418002071B595B0012269465B
S1131DF015A8FFF7FBF90400E4B2002C56D109A89A
S1131E0006903048079015996846FFF776F9040064
S1131E10E4B2002C4AD1059D002D01D1062403E033
S1131E20E87AC00700D5072429000098FEF7CFFC04
S1131E300600E4B2002C21D1E87AC0061ED5022E99
S1131E4001D202241AE0242269460CA8FEF750F9B4
S1131E500E9602210CA8FEF7ABFB0400E4B2002CA2
S1131E600CD100210CA8FEF755FE0400E4B2002CAE
S1131E7000D10724E4B2042C00D10024E4B2002CE5
S1131E8014D16846FEF767FF0400E4B2002C0DD1BC
S1131E90002E04D031000098FEF7FBFA0400E4B2EF
S1131EA0002C03D10098FEF795F904002000C0B27D
S1131EB016B070BD0000000052526141727241615F
S1131EC080180020D41200202DE9FC4104000F00EA
S1131ED0904600262500FFE7781E864213DA6B46FB
S1131EE0012201A94046FFF731FC009801280AD1DC
S1131EF09DF80400C0B20D28EED028706D1C761C2D
S1131F00C0B20A28E8D100202870002E00D1002495
S1131F102000BDE8F68130B583B004000D00E4B2C2
S1131F200A2C03D129000D20FFF7F5FF8DF800409E
S1131F30012401AB220069462800FFF7F2FC019856
S1131F40A04201D1012001E05FF0FF303EBD70B539
S1131F5004000D00002601E0641C761C2078002893
S1131F6009D029002078FFF7D6FF10F1010FF3D133
S1131F705FF0FF3000E0300070BD000010B582B0AB
S1131F8001220121DFF8F40700F0B7FD20215FF002
S1131F90402000F0E3FD202220215FF0402000F0EB
S1131FA0ACFD00240AE0FF21DFF8D40700F014FFA1
S1131FB06946DFF8CC0700F032FF641C0A2CF2D328
S1131FC020215FF0402000F0FDFD13BD00B583B07B
S1131FD0DFF8B00701F0FFF8DFF8AC0701F0FBF819
S1131FE0DFF8A80701F0F7F834215FF0402000F093
S1131FF0E9FD0121DFF8840700F0B0FD0A23022285
S113200034215FF0402000F0B9FC0A2302220121B0
S1132010DFF8680700F0B2FC01220121DFF85C0759
S113202000F06BFD01F056FA08210191DFF860170A
S11320300091002300220100DFF8440700F027FE8E
S1132040DFF83C0700F0A2FEFFF798FF07BD1CB5C0
S1132050DFF82C0700F0ADFE01F03CFA4408DFF88D
S11320603407844201D3DFF8304701F033FA082102
S113207001910094002300220100DFF8040700F01E
S113208006FEDFF8FC0600F081FE13BDDFF80C0746
S1132090007850F00100DFF804170870704780B52D
S11320A0C0B20100DFF8D80600F096FE6946DFF8FA
S11320B0D00600F0B4FE0098C0B202BD10B5040012
S11320C0FF20FFF7ECFF207010BD38B501F055FB81
S11320D010F5FA75FF20FFF7E2FF0400E4B2FF2CCD
S11320E003D001F04AFBA842F4D3E4B2FF2C01D19F
S11320F0012000E0002032BD80B501220121DFF87B
S11321007C0600F0FAFCFF20FFF7C9FF01BD80B593
S113211000220121DFF8640600F0EFFCFF20FFF746
S1132120BEFFFFF7D2FF002801D0012002E0FFF735
S1132130E3FF002002BDF8B504000D0001F01DFB13
S113214010F16407FF20FFF7AAFF0600F6B2FF2E86
S113215003D101F012FBB842F4D3F6B2FE2E01D043
S1132160002011E02000FFF7A9FF641C2000FFF706
S1132170A5FF641CAD1E002DF4D1FF20FFF78FFFD7
S1132180FF20FFF78CFF0120F2BD38B504000D00DD
S1132190FFF79BFF002801D1002024E02800C0B2F3
S11321A0FFF77DFFEDB2FD2D1CD04FF400752078B4
S11321B0FFF775FF641C2078FFF771FF641CAD1EE8
S11321C0002DF4D1FF20FFF76AFFFF20FFF767FF20
S11321D0FF20FFF764FFC0B210F01F00052801D0F4
S11321E0002000E0012032BD38B504000D002006B7
S11321F00AD514F07F0400213720FFF7F5FFC0B2A1
S1132200022801DBC0B23AE0FFF776FFFFF77FFF59
S1132210002801D1FF2032E054F04000C0B2FFF7A3
S11322203EFF280EC0B2FFF73AFF280CC0B2FFF7FA
S113223036FF280AC0B2FFF732FF2800C0B2FFF70A
S11322402EFF0125E4B2002C00D19525E4B2082C20
S113225000D187252800C0B2FFF721FFE4B20C2C7F
S113226002D1FF20FFF71BFF0A25FF20FFF717FF0E
S1132270010603D56D1EEDB2002DF6D1C0B232BDFC
S113228070B582B0C0B2002801D001209AE0DFF816
S11322900C050078800703D5DFF80005007891E08D
S11322A0FFF794FE00220121DFF8D00400F025FCA2
S11322B0002500210020FFF797FF012869D101F0D4
S11322C05CFA10F57A764FF4D5710820FFF78CFF8D
S11322D001283CD1002406E0FF20FFF7E0FE694618
S11322E0E4B20855641CE4B2042CF5DB9DF802004A
S11322F001284ED19DF80300AA284AD101F03DFAE5
S1132300B04206D25FF08041A920FFF76DFF00289C
S1132310F4D101F032FAB0423BD200213A20FFF767
S113232063FF002835D1002406E0FF20FFF7B7FE45
S11323306946E4B20855641CE4B2042CF5DB9DF84C
S11323400000400601D50C2523E0042521E00021EE
S1132350A920FFF749FF022802DA0225A92401E097
S11323600125012401F009FAB04206D2002120001F
S1132370C0B2FFF739FF0028F4D101F0FEF9B042F2
S113238006D24FF400711020FFF72EFF002800D072
S11323900025EDB2DFF808040560FFF7ADFEEDB2ED
S11323A0002D0AD0DFF8F403007810F0FE00DFF807
S11323B0EC130870FFF74BFE01E0FFF767FEDFF850
S11323C0DC03007876BDC0B2002801D0012002E011
S11323D0DFF8C8030078704738B50C0011001D0001
S11323E0C0B2002802D1EDB2002D01D104203FE09B
S11323F0DFF8A8030078C00701D5032038E0DFF830
S1132400A0030078000702D44FF400704143EDB2FA
S1132410012D0DD11120FFF7E7FE00281FD14FF445
S113242000712000FFF787FE002818D0002516E071
S11324301220FFF7D9FE002811D14FF400712000BB
S1132440FFF779FE002806D04FF4007004446D1E97
S1132450EDB2002DF1D100210C20FFF7C5FEFFF7EE
S11324604BFEEDB2002D01D0012000E00020C0B2EF
S113247032BD70B50C0015001E00C0B2002802D198
S1132480F6B2002E01D1042050E0C4480078C00701
S113249001D503204AE0C1480078400701D5022055
S11324A044E0BF480078000702D44FF4007045436D
S11324B0F6B2012E0DD129001820FFF795FE002851
S11324C02BD1FE212000FFF760FE002825D0002636
S11324D023E0B348007810F0060F04D0F6B23100C0
S11324E09720FFF781FE29001920FFF77DFE0028C1
S11324F013D1FC212000FFF748FE002806D04FF43A
S113250000700444761EF6B2002EF2D1FD210020A4
S1132510FFF73BFE002800D10126FFF7EDFDF6B2E0
S1132520002E01D0012000E00020C0B270BD30B503
S113253085B014002200C0B2002801D0042019E1A3
S113254096480078C00701D5032013E10125C9B2DC
S1132550002913D0012917D003295ED00A2900F0DD
S1132560BB800B2900F0BD800C2900F0C8800D2928
S113257000F0D3800E2900F0E380F6E0FFF7C7FDFA
S1132580002800D00025F1E000210920FFF72CFEEF
S1132590002841D110216846FFF7CDFD00283BD02B
S11325A09DF80000C0B28009C0B201280FD19DF887
S11325B009009DF8081010EB01209DF8071011F098
S11325C03F0110EB0140401C8002206023E09DF895
S11325D0050010F00F009DF80A10C9B210EBD110DD
S11325E09DF80910490011F006010818851C9DF892
S11325F00800C0B28009C0B29DF8071010EB81003A
S11326009DF8061011F0030110EB8120401CB5F178
S11326100901884020600025A8E06148007840074F
S113262020D500218D20FFF7DFFD002853D1FF20A6
S1132630FFF735FD10216846FFF77DFD00284AD0DD
S1132640302503E0FF20FFF72AFD6D1EEDB2002DBB
S1132650F8D110209DF80A10C9B2090988402060F9
S1132660002538E000210920FFF7BEFD002832D103
S113267010216846FFF75FFD00282CD048480078F9
S1132680800713D59DF80A00400010F07E009DF8E5
S11326900B10C9B2C909C9B20818401C9DF80D1025
S11326A0C9B28909491E8840206013E09DF80A00D8
S11326B0C0F38400C0B2401C9DF80B10C90011F097
S11326C018019DF80B20D2B25209D2B25118491CFC
S11326D048432060002549E0314800681070002517
S11326E044E000210920FFF77FFD002806D11021D6
S11326F02000FFF720FD002800D0002536E000214F
S11327000A20FFF771FD002806D110212000FFF7F1
S113271012FD002800D0002528E000213A20FFF710
S113272063FD00280BD1002505E0FF20FFF7B7FC6F
S1132730EDB260556D1CEDB2042DF6DB002515E0FD
S11327401748007840070FD500218D20FFF74CFD76
S1132750002809D1FF20FFF7A2FC40212000FFF749
S1132760EAFC002800D0002500E00425FFF7C4FCA3
S11327702800C0B205B030BD0A4870470070004060
S1132780008000401000001001000020080000201C
S1132790801A060021BCBE0020BCBE00010000203F
S11327A0481800200000AA4280B2802801DA010003
S11327B020E000290CD080B2FF2801DD002119E0BF
S11327C01B4980B201EB4000B0F58070018811E034
S11327D0002100E0491C89B2802907DA0200144B69
S11327E089B233F8113092B29A42F3D111F18000D8
S11327F000F0FF01080080B27047002100E0491C8E
S11328000C4A32F81120002A06D00200094B33F892
S1132810113092B29A42F2D1064A32F81120002ABB
S113282003D0054830F81100FFE780B2704700007C
S1132830E87300002870000008720000B0F1402F17
S11328405BD0DFF85013884257D0DFF84C1388422E
S113285053D0DFF8481388424FD0DFF8441388423E
S11328604BD0DFF84013884247D0DFF83C1388424E
S113287043D0DFF8381388423FD0DFF8341388425E
S11328803BD0DFF83013884237D0DFF82C1388426E
S113289033D0DFF8281388422FD0DFF8241388427E
S11328A02BD0DFF85813884227D0DFF8541388421E
S11328B023D0DFF8501388421FD0DFF84C1388422E
S11328C01BD0DFF84813884217D0DFF8441388423E
S11328D013D0DFF8401388420FD0DFF83C1388424E
S11328E00BD0DFF87013884207D0DFF86C138842EE
S11328F003D0DFF86813884201D1012000E00020F2
S1132900C0B2704770B504000D0016002000FFF738
S113291095FF002805D14FF49071DFF8440300F0CF
S11329203BFF002E09D0012E07D0022E05D04FF414
S11329309171DFF82C0300F02FFFF00705D514F593
S113294080600068EDB2284304E014F580600068FC
S1132950EDB2A84314F580610860B00705D514F5FD
S113296084600068EDB2284304E014F584600068D4
S1132970EDB2A84314F58461086070BDF8B5040095
S11329800D0017001E002000FFF758FF002805D196
S113299040F2FF11DFF8C80200F0FEFE012F0BD059
S11329A0022F09D0042F07D00C2F05D040F20321A9
S11329B0DFF8AC0200F0F0FE082E0DD00A2E0BD08A
S11329C00C2E09D0092E07D0002E05D04FF4027129
S11329D0DFF88C0200F0E0FEF80705D514F5A060DE
S11329E00068EDB2284304E014F5A0600068EDB27D
S11329F0A84314F5A0610860B80705D504F2045093
S1132A000068EDB2284304E004F204500068EDB21B
S1132A10A84304F204510860780705D514F5A160B1
S1132A200068EDB2284304E014F5A1600068EDB23B
S1132A30A84314F5A1610860380705D514F5A3600F
S1132A400068EDB2284304E014F5A3600068EDB219
S1132A50A84314F5A3610860F00705D504F20C50EF
S1132A600068EDB2284304E004F20C500068EDB2B3
S1132A70A84304F20C510860B00705D514F5A26010
S1132A800068EDB2284304E014F5A2600068EDB2DA
S1132A90A84314F5A2610860700705D504F2145028
S1132AA00068EDB2284304E004F214500068EDB26B
S1132AB0A84304F214510860300705D504F21C50F1
S1132AC00068EDB2284304E004F21C500068EDB243
S1132AD0A84304F21C510860002E05D114F5A5602A
S1132AE00068EDB2284304E014F5A5600068EDB277
S1132AF0A84314F5A5610860F1BD70B504000D008C
S1132B0016002000FFF79AFE002805D140F2853117
S1132B10DFF84C0100F040FEF6B2EDB214EB850094
S1132B20066070BD38B504000D002000FFF786FE76
S1132B30002805D140F25241DFF8240100F02CFEB8
S1132B4002222900C9B22000FFF7DCFE0823042278
S1132B502900C9B22000FFF711FF31BD38B50400C8
S1132B600D002000FFF76AFE002805D140F2F14174
S1132B70DFF8EC0000F010FE082301222900C9B29E
S1132B802000FFF7FBFE01222900C9B22000FFF755
S1132B90B9FE31BD00800540005000400090054062
S1132BA00060004000A005400070004000B00540F7
S1132BB00040024000C005400050024000D00540E3
S1132BC00060024038B504000D002000FFF736FE17
S1132BD0002804D140F29661214800F0DDFD022274
S1132BE02900C9B22000FFF78DFE08230122290025
S1132BF0C9B22000FFF7C2FE31BD000000E005406D
S1132C000070024000F0054000D003400000064080
S1132C1000100640002006400030064038B504008D
S1132C200D002000FFF70AFE002804D140F2EA61FB
S1132C300B4800F0B1FD02222900C9B22000FFF7C1
S1132C4061FE082301222900C9B22000FFF796FE85
S1132C5031BD0000004006400050064000600640C0
S1132C6074780000DFF8E41188420BD0DFF8E0113B
S1132C70884207D0DFF8DC11884203D0DFF8D8118E
S1132C80884201D1012000E00020C0B270472DE944
S1132C90F84304000F00150099462000FFF7E2FFF7
S1132CA0002804D1CC21DFF8B40100F075FD002D1B
S1132CB00ED0022D0CD0012D0AD0032D08D0102DDA
S1132CC006D0202D04D0D221DFF8900100F064FD5D
S1132CD0B9F1000F0AD0B9F1010F07D0B9F1020F11
S1132CE004D0D521DFF8740100F056FDDDF8208012
S1132CF0B9F1000F02D1780840450CD2B9F1000FA8
S1132D0004D00C20B7FBF0F0404504D2D721DFF803
S1132D104C0100F041FDB7FBF8F0B0F57E4F04D94B
S1132D20D821DFF8380100F037FD099E301F0D2847
S1132D3004D3D921DFF8240100F02EFDB9F1020FEC
S1132D4001D1082000E00020B9F1000F01D10021D9
S1132D5000E004210843211D0860B7FBF8F00021BE
S1132D60891CB0FBF1F2521EFF2AF9D814F11000AD
S1132D700160A80110F0C00015F0300550EA0220EF
S1132D802843711E08432060BDE8F18310B5040098
S1132D902000FFF767FF002804D14FF485712F4806
S1132DA000F0FAFC201D006850F00200211D0860AC
S1132DB010BD10B504002000FFF754FF002804D113
S1132DC040F22311254800F0E7FC201D006830F094
S1132DD00200211D086010BD38B504000D0020005C
S1132DE0FFF740FF002804D140F223211B4800F0E4
S1132DF0D3FC7FF00100216811F00F0188400542E7
S1132E0004D040F22521154800F0C6FC14F10C0052
S1132E1000688007FAD514F10800056031BD38B5A3
S1132E2004000D002000FFF71DFF002804D140F22C
S1132E307F210A4800F0B0FC14F10C000068400740
S1132E40FAD514F108000068286031BD0080004004
S1132E500090004000A0004000B00040D078000086
S1132E60DFF8E413884200F04A81DFF8E013884277
S1132E7000F04581DFF8D813884200F04081DFF884
S1132E80D413884200F03B81DFF8CC13884200F071
S1132E903681DFF8C813884200F03181DFF8C013AF
S1132EA0884200F02C81DFF8BC13884200F02781AF
S1132EB0DFF8B413884200F02281DFF8B0138842AF
S1132EC000F01D81DFF8A813884200F01881DFF8B4
S1132ED0A413884200F01381DFF89C13884200F0A9
S1132EE00E81DFF89813884200F00981DFF890130F
S1132EF0884200F00481DFF88C13884200F0FF80E0
S1132F00DFF88413884200F0FA80DFF880138842E7
S1132F1000F0F580DFF87813884200F0F080DFF8E5
S1132F207413884200F0EB80DFF86C13884200F0E1
S1132F30E680DFF86813884200F0E180DFF8601370
S1132F40884200F0DC80DFF85C13884200F0D78010
S1132F50DFF85413884200F0D280DFF8501388421F
S1132F6000F0CD80DFF84813884200F0C880DFF815
S1132F704413884200F0C380DFF83C13884200F019
S1132F80BE80402800F0BB80B0F1102F00F0B78065
S1132F90DFF82813884200F0B280DFF82413884257
S1132FA000F0AD80DFF81C13884200F0A880DFF841
S1132FB01813884200F0A380DFF81013884200F051
S1132FC09E80DFF80C13884200F09980DFF87C14AF
S1132FD0884200F09480DFF87814884200F08F80F3
S1132FE0DFF87014884200F08A80DFF86C1488429D
S1132FF000F08580DFF86414884200F08080B0F12E
S1133000101F7CD0DFF85814884278D0DFF85414AD
S1133010884274D0DFF85014884270D0DFF84C1422
S113302088426CD0DFF84814884268D0DFF8441432
S1133030884264D0DFF84014884260D0DFF83C1442
S113304088425CD0DFF83814884258D0DFF8341452
S1133050884254D0DFF83014884250D0DFF82C1462
S113306088424CD0DFF82814884248D0DFF8241472
S1133070884244D0DFF82014884240D0DFF81C1482
S113308088423CD0DFF81814884238D0DFF8141492
S1133090884234D0DFF81014884230D0DFF80C14A2
S11330A088422CD0DFF80814884228D0DFF80414B2
S11330B0884224D0B0F1202F21D0DFF8FC138842BD
S11330C01DD008281BD0DFF8F413884217D0DFF88E
S11330D0F013884213D0DFF8EC1388420FD0DFF8E6
S11330E0E81388420BD0DFF8E413884207D0DFF8F6
S11330F0E013884203D0DFF8D815884201D10120BB
S113310000E00020C0B2704710B582B00400200077
S1133110FFF7A6FE002805D140F23131DFF8AC05F7
S113312000F03AFB14F07040B0F1704F25D1C4F3B5
S11331300720DFF8A0150818A10011F47F7151EAE7
S1133140401050F08440012101600020009002E012
S11331500098401C009000981028F9D3C4F307206D
S1133160DFF870150818A10011F47F7151EA4010BE
S113317050F08440002101602CE0DFF86005210F4D
S113318050F821000068A1B2220C12F01F029140F5
S11331900843DFF84815220F51F822100860002078
S11331A0009002E00098401C009000981028F9D389
S11331B0DFF82805210F50F821000068A1B2220C85
S11331C012F01F0291408843DFF81015220F51F8C6
S11331D02210086013BD10B504002000FFF740FE64
S11331E0002805D140F29631DFF8E00400F0D4FA6B
S11331F014F07040B0F1704F0ED1C4F30720DFF823
S1133200D8140818A10011F47F7151EA401050F04D
S113321084400121016011E0DFF8C404210F50F85B
S113322021000068A1B2220C12F01F029140084351
S1133230DFF8AC14220F51F82210086010BD000012
S11332400138FDD1704770470100100002001000E2
S11332500001100000021000000410000001101012
S11332600002101000041010005800F0004010106C
S113327000501020005400F0010000200200002043
S1133280040000200800002010000020200000207E
S1133290400000208000002000010020090800F008
S11332A00A0800F00B0800F00C0800F00D0800F00C
S11332B00E0800F00F0800F0100800F000400010A5
S11332C0022000F0032000F0042000F0052000F0AC
S11332D00010101070B50400DFF81404006810F03A
S11332E0E04F08D0DFF808040068DFF8081408404D
S11332F0B0F1805F02D1002C00F1A780DFF8E40375
S11333000568DFF8F403066855F4006535F48005B4
S113331056F40066DFF8CC030560DFF8DC030660D2
S1133320A80701D5A00708D515F0010014F0010184
S113333091F00101C0B208421ED074F003000540B0
S1133340DFF8A0030560002E07D516F070003028C2
S113335009D016F07000702805D0002E08D415F09E
S11333603000302804D14FF48050FFF769FF03E0A8
S11333705FF40020FFF764FF35F4FE6514F4FE608B
S11333800543DFF878030640DFF874032040064362
S1133390E00010F040000643DFF848030560DFF862
S11333A0580306601020FFF74BFF35F4405514F422
S11333B04050054336F4005614F4005006434020B0
S11333C0DFF824130860002E06D5DFF82C0306600E
S11333D0DFF81003056005E0DFF808030560DFF897
S11333E018030660DFF81C030540DFF81C032040C7
S11333F0054336F0FC5614F0FC500643600008D533
S113340055F4800536F48006DFF8000320400643B7
S113341001E036F0804620050ED44FF4004000E071
S1133420401E002804D0DFF8C41209684906F7D505
S113343035F4006536F40066DFF8A8020560DFF8AD
S1133440B80206601020FFF7FBFE70BD00011020DB
S1133450004800F080000030005000F01000003000
S1133460014000F0000100100002001010000010E4
S113347020000010021C00F0031C00F020000030AB
S113348001001010020010100400101008001010A9
S1133490040400F0050400F0010000100200001014
S11334A004000010031800F0041800F0051800F0E0
S11334B0061800F0071800F001001020001010009A
S11334C0005C00F0015C00F0025C00F0035C00F0C2
S11334D0045C00F030B4DFF80C020168DFF8180275
S11334E00268002A02D512F0700001E011F03000E9
S11334F000280DD010283AD020286FD0302800F0B2
S1133500A480602800F0A480702800F0A480A5E0C6
S1133510DFF8FC01C1F3841350F82300DFF8F43121
S11335201340B3F1004F05D0002A00F1AA800B0527
S113353000F1A780DFF8E0311B68DFF8B4412468AC
S113354014F0E04F09D0DFF8A8412468DFF8A45153
S11335502C40B4F1805F40F08380C3F34814A41C72
S1133560604313F01F04A41CB0FBF4F081E0DFF807
S11335708001006810F0E04F08D0DFF874010068A3
S1133580DFF870311840B0F1805F02D1DFF88C01B0
S113359023E0DFF85C010068DFF858311840DFF8F9
S11335A08031984205D1DFF84801006880B20228D2
S11335B00ED0DFF83C010068DFF838311840DFF83E
S11335C06431984207D1DFF828010068000402D171
S11335D0DFF8540101E0DFF854019FE7DFF8100140
S11335E0006810F0E04F08D0DFF804010068DFF84D
S11335F004311840B0F1805F02D1DFF8340123E0D8
S1133600DFF8EC000068DFF8EC301840DFF8103128
S1133610984205D1DFF8D800006880B202280ED0A5
S1133620DFF8CC000068DFF8CC301840DFF8F43065
S1133630984207D1DFF8B8000068000402D1DFF82F
S1133640F40001E0DFF8F00068E747F2305065E786
S11336505FF4800062E74FF400405FE7002032E04F
S1133660C3F34814604313F01F04641C6400B0FBEC
S1133670F4F05C0400D540081B0400D5800851F424
S113368080014B021FD5002A18D5530010D5DFF84E
S113369084301340B3F1004F03D0002A08D4090545
S11336A006D44000C2F38651491CB0FBF1F00AE095
S11336B0C2F3C551491CB0FBF1F004E0C1F3C3519E
S11336C0491CB0FBF1F030BC704700005477000097
S11336D0055C00F000E50F4000E60F40487D000067
S11336E0547D000060E00F4058E00F4050E00F4070
S11336F000E00F400000FF7070E00F408FFFFF7F7D
S113370030000080FCFF3FF80300C0070000404089
S1133710287600000008008064E00F40C0E1E40067
S11337200000011000000310001BB7000024F40087
S113373070383900C0C62D0000093D0080B500F086
S11337400EF84CF24F301049086000200F49086011
S113375005200F49086000200E49086001BD0020C3
S11337600B49086070470A480068C00304D509483B
S11337700068401C07490860704780B5FFF7F3FFF5
S11337800448006802BD000014E000E018E000E016
S113379010E000E05418002080B500F002F8FCE7C7
S11337A070477047C2788A18DFF81832DA70837865
S11337B00A0092B2120AD218DFF808329A704278DC
S11337C0DFF800325A700078DFF8F8211070DFF863
S11337D0F4018278080080B2000A80B2824212DAD0
S11337E0DFF8E0014078401CDFF8D8215070DFF8A2
S11337F0D4014078002806D1DFF8C8010078401CC5
S1133800DFF8C0211070DFF8BC01C07889B201F084
S1133810FF01884217DADFF8AC018078401C69495F
S113382088706848807800280DD166484078401C2C
S11338306449487063484078002804D1614800789E
S1133840401C60490870704710B492B20A44531E79
S11338500BE00A784C7814EB022210180400A4B28E
S113386092B2944200D2401C891C9942F1D39942ED
S113387008D109780A021018010089B292B2914263
S113388000D2401C80B210BC704780B514224E494F
S11338900020FFF7D9FF80B2002802D14FF6FF7055
S11338A002E080B201F076F880B202BD10B547495B
S11338B0097C464A527C12EB0121B1F11404C0B2D6
S11338C000190822424980B2FFF7BEFF220092B2DB
S11338D0404980B2FFF7B8FF80B2002802D14FF60A
S11338E0FF7002E080B201F055F880B210BD80B5DF
S11338F00620FFF7DBFF02BD0020374908700AE00D
S113390000203649344A127821F8120032480078EF
S1133910401C31490870304800780028F0D000205D
S11339202D4908700CE000202D492B4A1278682399
S11339305A431144487628480078401C26490870A8
S1133940254800780028EED04FF48060254908808F
S113395070470021204A117004E01F490978491C6E
S11339601D4A11701C49097800290CD11B491A4AB7
S1133970127831F812100029EFD11849164A12783A
S113398021F81200FFE7704780B5010089B216489C
S113399000680830FFF706FF0A48007812490968F2
S11339A008720848407810490968487205488078C8
S11339B00D49096888720348C0780B490968C872C0
S11339C001BD000078180020160200200802002023
S11339D0220200202A0200209318002086180020CA
S11339E0581600208A1800207018002010B5DFF83F
S11339F0AC1D0C68DFF8F81DDFF8F82D1160DFF856
S1133A00F41D0968DFF8F02D1160C0B2032818D145
S1133A10607E10F00F0003280AD1208A002807D105
S1133A200820DFF8D81D087001F05BF800F07ABEBA
S1133A300020DFF8CC1D08800020DFF8C01D0870CE
S1133A4010BDC0B2022840F0D180DFF8B80DC078B4
S1133A50401CDFF8B01DC870DFF8A80DC07800283E
S1133A601ED1DFF8A00D8078401CDFF8981D887007
S1133A70DFF8900D8078002812D1DFF8880D4078A7
S1133A80401CDFF8801D4870DFF8780D407800286E
S1133A9006D1DFF8700D0078401CDFF8681D08704F
S1133AA00020DFF85C1D08800020DFF85C1D088022
S1133AB0607E072802D0607E052808D1A07E401CC5
S1133AC0A076A07E782801D100206076B0E7607EE1
S1133AD00028FBD0208A00287AD0A07E411EA1763F
S1133AE0C0B20028F2D1E07E082808D0607E022807
S1133AF002D0607E012810D1E07E05280DD100207F
S1133B0060768020DFF8F41C087000F0EAFF1420CF
S1133B10DFF8C41D81F82F008DE1E07E052801DB6C
S1133B20042000E0E07E032111FA00F0A076E07E9C
S1133B30401CE076607E10F00F00C0B201280AD06D
S1133B40022835D0032839D004283FD006283DD098
S1133B5008283BD0BAE71020DFF87C1D81F82F003D
S1133B60DFF8740D90F82F0050F00200DFF8681DA4
S1133B7081F82F000220DFF8601D81F83600042050
S1133B80DFF8541D81F837000620DFF84C1D81F85A
S1133B9038000A20DFF8401D81F839002C20DFF8B6
S1133BA0601C08806020DFF8301D81F82E004BE196
S1133BB00020DFF8241D81F82F00D1E70420DFF86E
S1133BC03C1C087000F08DFF00F0EFBD00F051BD0B
S1133BD0607E10F00F0003287FF478AF0820DFF830
S1133BE01C1C087000F07DFF00F09CBDDFF8E80CA1
S1133BF0807B45287FF41CAFDFF8040C0088DFF8D5
S1133C00D81C097CDFF8D02C527C12EB01218842AD
S1133C1016DBDFF8C40C007CDFF8BC1C497C11EB1C
S1133C200020DFF8DC1B0880DFF8AC0C007D3F21AE
S1133C30084204D1DFF8A00C407D002801D0F7E64B
S1133C40F6E6DFF8840D0088DFF8801D09888842D5
S1133C5007D1DFF8740D4088DFF8701D4988884269
S1133C6010D0DFF8740CC08BDFF85C1D0988884223
S1133C7007D1DFF8640C008CDFF84C1D49888842BA
S1133C8000D0D5E6FFF701FE4FF6FF7188427FF4BE
S1133C90CFAEDFF8440CC07D062808D1FFF727FE1D
S1133CA04FF6FF71884244D1DFF8244D43E0DFF83A
S1133CB0280CC07D01287FF4BBAEDFF81C0C90F803
S1133CC0220008287FF4B4AE0020DFF80C1C81F831
S1133CD02200DFF8040C808C4FF6F771884207DB72
S1133CE0DFF8F40B808C0930DFF8EC1B888406E0E5
S1133CF0DFF8E40B808C0830DFF8DC1B8884DFF805
S1133D00D80B408BDFF8D01BC883DFF8CC0B808B3B
S1133D10DFF8C41B0884DFF8B00C0088DFF8B81B98
S1133D204883DFF8A40C4088DFF8AC1B888300F0DC
S1133D302CBE7DE66834DFF8980CA042C0F0DF802A
S1133D40607E0028F6D0DFF8900B808CA188884232
S1133D50F0D1DFF8840B408CE1888842EAD1DFF8A7
S1133D60780B408B21888842E4D1DFF86C0B808B80
S1133D7061888842DED1DFF8240A04600020DFF87D
S1133D807C1A0870DFF8500B90F82F00400700F100
S1133D90CC82DFF8440B90F82E00C0B200098000FA
S1133DA0DFF8301C0870DFF8580A0088DFF8241C9C
S1133DB00978401A1438DFF8481A0880607E10F039
S1133DC00F00022808D1DFF8100B90F82F0010F034
S1133DD03F00122800F0B382DFF8240A008800288C
S1133DE007D1DFF8F40A90F82F000321084200F00D
S1133DF0A682DFF8E40A90F82600217A884215D1D9
S1133E00DFF8D40A90F82700617A88420ED1DFF8EF
S1133E10C80A90F82800A17A884207D1DFF8B80AC6
S1133E2090F82900E17A884200F089821020DFF8B6
S1133E30A81A81F82F002820DFF8C4190880502020
S1133E40DFF8941A81F82E00207ADFF88C1A81F8B2
S1133E502A00607ADFF8801A81F82B00A07ADFF854
S1133E60781A81F82C00E07ADFF86C1A81F82D00BA
S1133E70207BDFF8641A81F82600607BDFF8581A8B
S1133E8081F82700A07BDFF8501A81F82800E07B36
S1133E90DFF8441A81F829000620DFF83C1AC875B7
S1133EA0A088DFF8341A4884E088DFF82C1A888464
S1133EB0DFF8140B0088DFF8201A4883DFF8080BBA
S1133EC04088DFF8141A88832088DFF80C1AC88326
S1133ED06088DFF8041A0884607EC00640F10A8511
S1133EE00020DFF8F41981F83100DFF8EC0990F8CC
S1133EF03100DFF8E41981F8300000F003BDDFF889
S1133F00D80990F82F0010F03F00022806D0DFF8FF
S1133F10C80990F82F00400729D589E5DFF8B809CA
S1133F20808CDFF8B41A08800020DFF8A81A087023
S1133F3006E0DFF8A00A0078401CDFF8981A087041
S1133F40DFF8900A00780028E1D1DFF88C0A0088B5
S1133F50DFF8881ADFF87C2A127831F812108842C8
S1133F60E7D100240020DFF86C1A0870F0E0142078
S1133F70DFF8641981F82F002820DFF884180880FE
S1133F805020DFF8541981F82E00DFF84C0990F81E
S1133F902900DFF8401A0870DFF83C0990F82D007A
S1133FA0DFF8341981F82900DFF8280A0078DFF8EF
S1133FB0281981F82D00DFF8200990F82800DFF88F
S1133FC0141A0870DFF8100990F82C00DFF80819AB
S1133FD081F82800DFF8FC090078DFF8FC1881F884
S1133FE02C00DFF8F40890F82700DFF8E8190870CF
S1133FF0DFF8E40890F82B00DFF8DC1881F82700DC
S1134000DFF8D0090078DFF8D01881F82B00DFF84A
S1134010C80890F82600DFF8BC190870DFF8B80863
S113402090F82A00DFF8B01881F82600DFF8A40918
S11340300078DFF8A41881F82A00DFF89C0890F8CB
S11340402D00401CDFF8901881F82D00DFF8880857
S113405090F82D00002826D1DFF87C0890F82C0079
S1134060401CDFF8741881F82C00DFF86C0890F815
S11340702C00002817D1DFF8600890F82B00401CB2
S1134080DFF8541881F82B00DFF84C0890F82B0067
S1134090002808D1DFF8400890F82A00401CDFF817
S11340A0381881F82A00DFF83008408CDFF8281926
S11340B00880DFF82408808CDFF81C184884DFF8B7
S11340C018090088DFF810188884DFF80C08408B82
S11340D0DFF80418C883DFF80008808BDFF8F817CE
S11340E00884DFF8E4080088DFF8EC174883DFF879
S11340F0D8084088DFF8E017888300F003BCDFF8B5
S1134100D008DFF8D0180978682251430844407E6B
S1134110072816D1002C0BD0A07EDFF8B418DFF8E6
S1134120B428127868235A431144897E884208D2FD
S1134130DFF89C08DFF89C1809786822514300EBEB
S11341400104DFF890080078401CDFF88818087034
S1134150DFF880080078002813D1DFF87408DFF84E
S113416074180978682251430844407E0028C6D157
S1134170DFF85C08DFF85C1809786822514300EB2B
S11341800104002C3FF454ACDFF810060460032053
S1134190A076A07E20760020A0750420E075002083
S11341A0E076DFF83407808CA080DFF82C07408CA1
S11341B0E080DFF82407408B2080DFF81C07808B29
S11341C0608001206076DFF83C0600782073DFF819
S11341D0340640786073DFF82C068078A073DFF82B
S11341E02406C078E07301202082DFF8EC0690F802
S11341F02900E072DFF8E00690F82800A072DFF8EA
S1134200D80690F827006072DFF8CC0690F82600F4
S113421020720120FFF7B8FBDFF8BC0690F82E00EF
S113422010F0F0005128FFF696AC0020DFF8A41738
S1134230087006E0DFF89C070078401CDFF894174C
S11342400870DFF890070078DFF88C1691F82E10CC
S1134250C9B20909C9B2491FB0EB810FBFF67BACE3
S1134260DFF87406DFF86C170978084490F8360014
S1134270DFF86C170870DFF86807007800283FF44F
S11342806AACDFF85C0700780128D3D0DFF8500768
S1134290007802282ED1DFF84006DFF838170978B5
S11342A0084490F83700042824D1DFF82C06DFF8FE
S11342B024170978084490F83800DFF81C16DFF852
S11342C014271278114491F8391051EA0020DFF8CC
S11342D008170880DFF80007008840F20B61884265
S11342E002DB40F20A6002E0DFF8EC06008860823C
S11342F0A08230E4DFF8E005DFF8D8160978084436
S113430090F8370000283FF426ACDFF8C8060078A0
S1134310DFF8C415DFF8BC261278114491F8371081
S11343200818DFF8B01608708BE7002060762020AC
S1134330DFF8C814087000F0D4FBFFF779BBDFF88E
S1134340980590F82F00C00664D5208A002861D013
S1134350218A14F10C00FFF725FADFF87C0590F8A8
S11343602A00DFF880160978884253D1DFF86805FF
S113437090F82B00DFF86C16497888424AD1DFF8B0
S1134380580590F82C00DFF85C168978884241D1F2
S1134390DFF8440590F82D00DFF84816C978884204
S11343A038D1DFF8400600782073DFF8380640780B
S11343B06073DFF830068078A073DFF82806C078D1
S11343C0E073E07E00281DD194F9180094F91A10C6
S11343D0401AA17DC9B2B0EBD100A17D4118A175ED
S11343E040B2002801D540B24042E17DC9B2B0EBF1
S11343F09100E17D4018E075A07DC0B2E17D11EB34
S1134400D00020760120DFF8F4130870207EA07617
S113441000202082607E10F00F00C0B2012813D06B
S1134420C0F06682032800F0FA8035D3052800F036
S11344303082C0F0F981072800F05082C0F0508229
S1134440082800F0E58153E2DFF8B0030078C007E4
S113445020D5032060764020DFF8A01308700020E8
S11344602082DFF89C03008800280CD0DFF88C033E
S1134470007850F00200DFF884130870DFF880033E
S11344800088FFF781FA0020DFF87C13088000F031
S113449028FB47E1FFF7CCBADFF860030078C007D8
S11344A040F1B380DFF8300490F82F0010F03F00A3
S11344B0122840F0AA80DFF8200490F82E0010F0B3
S11344C0F000512829DB0020DFF80815087006E009
S11344D0DFF800050078401CDFF8F8140870DFF8F6
S11344E0F4040078DFF8F01391F82E10C9B209092A
S11344F0C9B2491FB0EB810F0FDADFF8DC03DFF834
S1134500D4140978084490F83600DFF8D4140870FD
S1134510DFF8CC040078002826D103206076DFF889
S1134520B80390F826002072DFF8AC0390F8270057
S11345306072DFF8A40390F82800A072DFF89803F3
S113454090F82900E0720120FFF71EFA4220AB49DF
S11345500870002020820020A94908800020AA4970
S1134560088000F0BEFADDE0DFF87404007801286A
S1134570AED0DFF86C04007802282ED1DFF858039F
S1134580DFF850140978084490F83700042824D13F
S1134590DFF84403DFF83C140978084490F8380045
S11345A0DFF83413DFF82C241278114491F8391011
S11345B051EA0020DFF820140880DFF81C0400888A
S11345C040F20B61884202DB40F20A6002E0DFF84D
S11345D0080400886082A0829FE7BF48DFF8F413D4
S11345E00978084490F83700002896D0DFF8E403EF
S11345F00078B949DFF8DC231278114491F83710B8
S11346000818DFF8D013087069E720207B49087088
S113461000F067FA002061490968487677E4AE48FB
S113462090F82F00C0072AD5607EC00627D4208AC0
S113463000287FF4FDA972480088401C80B2FFF76F
S1134640A3F96E48007850F010006C4908706C486B
S11346500088002805D06948007850F002006749B6
S1134660087000F03EFA01202082082060760020C5
S1134670E0761120984981F82F00FFF7DCBB9648BB
S113468090F82F00800619D55A480068924991F88D
S11346903410914A92F8352052EA012108445549D0
S11346A00860574800888C4991F834108A4A92F877
S11346B0352052EA0121401A5149088050480088A7
S11346C000280CD0607EC00609D44C48007850F015
S11346D002004A4908704A480088FFF755F97E48A5
S11346E090F830007C4991F8311011EB0020BA4960
S11346F00880A08AB8490988884203D3B64800884C
S1134700002802D1A08AB4490880B3480088608296
S11347103A4800780321084278D000203A490880BA
S113472000F0DFF93548007880060AD500203649C4
S11347300880002060761420674981F82F00FFF775
S11347407ABB2E480078C0060ED500202E4908807A
S113475001202082042060760020E07611205E494A
S113476081F82F00FFF767BB2748008800281AD07C
S113477022480078C00701D500202082208A002822
S11347800ED1608A20490988884202D2608A1E4973
S113479008801D480088208205E000BF70180020B2
S11347A0208A194908800020E076134800681149DE
S11347B008601548008800280CD0208A002809D0F9
S11347C0208A28300E4908801820434981F82F0098
S11347D0FFF735BB09480078800717D5282008491A
S11347E0088010203C4981F82F00FFF728BB00BF48
S11347F03E020020681800206C1800209218002047
S1134800821800207418002084180020FFF710B9C3
S113481075480078C00706D50020607610207249DC
S1134820087000F05EF963E070480088002803D047
S11348306E480088FFF7A8F8274890F82F00C007B3
S113484016D569480078C00706D507206076002091
S1134850A0760020208201E0062060760120FFF788
S113486093F810206049087000F03BF9FFF7DEBAB6
S11348705D480078C00705D50520607600202082B9
S1134880FFF7D6B85948008800287FF4CFAAFFF76D
S1134890CFB856480088002803D054480088FFF752
S11348A073F80D4890F82F00C0070DD507206076E7
S11348B00020A0760120FFF767F810204A4908700D
S11348C000F00FF9FFF7B2BA4848008800287FF4D7
S11348D0ADAAFFF7ADB800BF08020020FFF7A6BAE3
S11348E041480078C00703D5072060760020A076F1
S11348F0FFF79EB806203E4981F830000A203C4963
S113490081F8310040203A4988753848008880B2DF
S1134910000A37490874354800883549487400202E
S1134920334981F83500324890F83500304981F830
S1134930340000202E494886FEF7D9FFC0432C4995
S1134940488645202A49887300202949C8730020D5
S1134950274948752648407D25490875254800881B
S1134960401C244908802348008880B2000A20495A
S11349708874204800881E49C87400201C49088394
S1134980FEF783FFC0431A490883002016490870C4
S1134990FFF756B8010089B2090A51EA002080B233
S11349A0704710B501290DDB134A118013490968BA
S11349B0884207D010490A8810490C680100200079
S11349C000F03EF910BD00005C180020947D00004A
S11349D058160020931800208C18002086180020F8
S11349E094180020781800209218002082180020C3
S11349F00802002088180020841800206C18002069
S1134A0080B500F059F9FEF7B8FE10F5FA70814947
S1134A100860FEF7B2FE00F51C5010307E490860B5
S1134A20FEF76AFF4FF6A960ADF8000043F6137075
S1134A30ADF80200BDF8000078490880BDF8020016
S1134A40764948804FF6FF70ADF800000020ADF8BD
S1134A500200BDF8000072490880BDF802007049E8
S1134A6048804FF6A960ADF8000040F21310ADF88D
S1134A700200BDF800006B490880BDF802006949D6
S1134A8048804EF60300FEF764FF00F01DF901BDF7
S1134A9038B5654A126812F11C042268626000226B
S1134AA006E092B2835C92B204EB02052B72521CB4
S1134AB013000D00EDB29BB2ADB2AB42F1D3C9B25B
S1134AC0081DA4F84800B4F84810201DFFF769FF3A
S1134AD02068401C206031BD80B500F032F8002011
S1134AE002BD10B55048006810F11C044F4800780E
S1134AF0400605D5012020600020A4F848001FE0EE
S1134B004A480078C00702D50020A4F84800474866
S1134B100078400708D5B4F84800002804D0B4F859
S1134B204810201DFFF73DFF40480078800707D557
S1134B300020A4F848003E480068001D00F0A4F9D5
S1134B4010BD10B500F04AF900282DD0394908806D
S1134B504FF40060FFF71EFF3749898980B2814214
S1134B600ED10120FEF742FF3248008800281BD0F6
S1134B7000F0EAFC00F047F900202E49088013E019
S1134B8040F60600FFF706FF2B49898980B281426F
S1134B900AD100F06FFC27480088002804D000F0F8
S1134BA032F9002023490880FEF7E7FD1949096816
S1134BB088421FD31748006810F5FA701549086039
S1134BC0002415E01D48682101FB04F1084416493E
S1134BD008600220FEF70AFF16480088002806D065
S1134BE000F0B2FC00F00FF9002012490880641CA8
S1134BF0002CE7D0FEF7C1FD07490968884208D3B5
S1134C000548006800F51C5010300349086000F0A6
S1134C105BFB10BD4C180020501800205C180020CD
S1134C2064180020601800207018002092180020DA
S1134C30681800208218002008020020581600205E
S1134C4062B38B0708D0521E11F8013B00F8013BF8
S1134C5000F024808B07F6D1830740F0208000BF4A
S1134C60103A07D330B4B1E83810103AA0E838103D
S1134C70F9D230BC530724BFB1E80810A0E80810EB
S1134C8044BF51F8043B40F8043BD20724BF31F839
S1134C90022B20F8022B44BF0B7803707047083AAC
S1134CA007D3B1E80810083A40F8043B40F804CBB5
S1134CB0F7D25307E4E7000080B55748FEF78BFAB4
S1134CC05548FEF721FA01BD30B585B05348FEF7CB
S1134CD082FA0C215248FDF725FF7F21514800F04C
S1134CE0A8FE00214F4800F0BEFE040021004D48FC
S1134CF000F0CCFEFEF7EEFB01004A4800F004FD94
S1134D001621484800F017FD464800F079FD0121BE
S1134D10444800F0D1FE0400FEF72FFD00F598553D
S1134D208835600708D401213E4800F0C5FE040020
S1134D30FEF723FDA842F4D308208DF800000020DC
S1134D408DF8010027208DF8020069208DF80300FA
S1134D505B208DF8040045208DF8050002A903A806
S1134D6000F064FF039810F1010F19D0029810F1BC
S1134D70010F15D003988DF800000398000A8DF8F0
S1134D8001000398000C8DF8020002988DF80300CE
S1134D900298000A8DF804000298000C8DF80500B2
S1134DA06946204800F0FEFC9DF800001E4908708A
S1134DB09DF801001C4948709DF802001A4988704A
S1134DC09DF803001849C8709DF80400164908713D
S1134DD09DF805001449487105B030BD10B5002197
S1134DE0104800F040FE040021000E4800F04EFE82
S1134DF0E00706D540F242620C490A4800F07AFD09
S1134E0000E0002010BD80B5094802880749054824
S1134E1000F0EAFD01BD0000005010202000002039
S1134E20005002400080044038180020080200208E
S1134E30821800200020DFF8701408700020DFF8CA
S1134E40681488640020DFF8601481F843000020AF
S1134E50DFF85414A1F844000020DFF84C148870E3
S1134E600020DFF8441448707047DFF83C040078F1
S1134E70002801D1002000E0012070470020DFF865
S1134E80281481F84300704780B50178FF291ED1AA
S1134E9000F091F8DFF8100490F84300012802D1E3
S1134EA0102000F07EF8DFF80004B0F94400012877
S1134EB00CDB0120DFF8F01381F84300DFF8E8038E
S1134EC0B0F94410DFF8E40300F053F801BDDFF853
S1134ED0D813097801294BD10178C92932D0CC29BA
S1134EE03FD0CF293AD0D0292FD0D12933D0D229BD
S1134EF02ED0F32917D0F4290FD0F5290AD0F6299A
S1134F000ED0FA2912D0FC2913D0FD2914D0FE2981
S1134F1015D029E000F0D9F8BCE700F0F9F8B9E7BA
S1134F2000F0C8F8B6E700F019F9B3E700F0AAF802
S1134F30B0E700F0A2F8ADE700F087F8AAE700F0C8
S1134F4076F8A7E700F03DF9A4E700F05CF9A1E7E3
S1134F5000F01BF99EE700F088F99BE700F099F94F
S1134F6098E700F0ABF995E7202000F01AF891E7F4
S1134F70ACE780B589B200F0C8FE01BD10B40023CF
S1134F8002E00478E318401C0C00611E002CF8D1E8
S1134F90DBB21360012010BC70470020C249487086
S1134FA07047FE21C04AD170BF4908710220BE4932
S1134FB0A1F84400704780B500F005FF002803D134
S1134FC01020FFF7EEFF31E0FFF7E7FF0120B649BD
S1134FD00870FF20B449C8700020B3490871B24872
S1134FE0007950F01000B04908710020AE494871B2
S1134FF0AD484079AC49487100F09FFEAA498871D8
S113500000F0B0FEA849C87100F0ACFE80B2000AFE
S1135010A54908720120A44948720120A249887256
S11350200820A149A1F8440001F089FA01BD80B526
S113503000209D490870FFF7B0FFFF209A49C8700F
S113504001209949A1F8440001BDFF209649C87088
S1135050002095490871944840789349487100208C
S11350609149887100209049C87100208E490872C6
S113507006208D49A1F84400704780B50020FFF751
S113508090FF01BDFF208849C8708948864988641B
S11350900020854908710020834948710020824915
S11350A0887107208049C1F8070008207E49A1F8CB
S11350B044007047FF217C4AD17040687A49886473
S11350C001207949A1F84400704710B5040000F0AC
S11350D034FE80B2401E6178884203DA2220FFF752
S11350E060FF14E0627892B26F48816C714801F0FD
S11350F065FAFF206C49C8706B48806C61780818A9
S1135100694988646078401C6749A1F8440010BD6F
S113511010B5040000F011FE80B2401E6178884290
S113512003DA2220FFF73DFF17E060685E498864D8
S1135130627892B25C48816C5E4801F03FFAFF20CD
S11351405949C8705848806C617808185649886471
S11351506078401C5449A1F8440010BD80B5FF217B
S1135160514AD170544A41684F48806CFFF706FF9A
S11351704D49087100204C49487100204A49887102
S113518008204949A1F8440001BD80B5FF204649E3
S1135190C87000204449087100204349487100F058
S11351A0CCFD4149887100203F49C87100203E4927
S11351B0087200203C49487207203B49A1F844008A
S11351C001BD10B5040000F0B8FD621C80B2411EA0
S11351D03548806C01F0B7F9002803D13120FFF77E
S11351E0E0FE0FE0FF203049C87000F0A6FD2E4914
S11351F0896C80B2401E40182B49886401202A49DA
S1135200A1F8440010BD10B5040000F096FD80B272
S1135210801E6178884203DA2220FFF7C2FE23E071
S1135220FF202149C87001201F49A1F8440060787B
S1135230002807D101F097F9002802D13120FFF7A7
S1135240B0FE11E0A21C61781748806C01F07BF974
S1135250002803D13120FFF7A4FE05E01248806C3A
S1135260617808181049886410BD80B541680E48FB
S1135270806C01F06CF9002803D13120FFF791FE16
S113528006E0FF200849C87001200749A1F844003E
S113529001BD80B501F076F9FF200349C8700120F3
S11352A00149A1F8440001BD201700202317002064
S11352B08C7D0000241700202717002080B53120A2
S11352C0FFF76FFE01BD000010B5DFF8F4030078AE
S11352D0401CDFF8EC1308700020DFF8DC130870C2
S11352E020E0DFF8D803DFF8D01309780C2251430B
S11352F000EB010420886188084300280BD0DFF804
S1135300C0030078A17A401A782804DB0421002223
S1135310200001F065F9DFF8A0030078401CDFF8F5
S113532098130870DFF8900300780828D9DB10BDC3
S113533070B50C000021DFF88023117006E0DFF85F
S113534078130978491CDFF870231170DFF86813AB
S11353500978082921DADFF86413DFF85C2312786E
S11353600C235A4301EB020529880029E7D06988F8
S11353700029E4D001882A889142E0D141886A88D2
S11353809142DCD106222E1D21003000FFF758FC8B
S1135390DFF82C030078A8726BE00021DFF81823F3
S11353A0117006E0DFF810130978491CDFF80823B0
S11353B01170DFF80413097808290EDADFF8FC12FB
S11353C0DFF8F42212780C235A4301EB02052988F2
S11353D00029E7D169880029E4D1DFF8DC120978D3
S11353E0082938D10021DFF8DC2211700021DFF810
S11353F0D82211700021B04A11701DE0AF49AE4AA5
S113540012780C235A4301EB0205AE490978AC4AE1
S11354101278AB7AD21A914209DAA9490978AA7AA0
S1135420891AA84A1170A4490978A74A1170A24997
S11354300978491CA04A11709F4909780829DDDBC5
S1135440A14909789C4A11709C499B4A12780C2303
S11354505A4301EB0205042201002800FFF7F0FB88
S113546006222E1D21003000FFF7EAFB9448007845
S1135470A87270BD10B5954800882A2803D2002070
S1135480924908805FE00020904908809048808A13
S1135490B0F5807F03D0B0F5007F44D053E08C4852
S11354A0C08C8C49098888423CD18948008D89493F
S11354B04988884236D188498848FFF739FF4FF434
S11354C000708349888206228349854C2000FFF7B7
S11354D0B7FB06228349804C2000FFF7B1FB06226C
S11354E08049814C2000FFF7ABFB06227C49784CB5
S11354F02000FFF7A5FB7648808B7549C884744863
S1135500C08B734908857348008871498883714842
S113551040886F49C8834FF4C1606D4988812A204F
S11355206A4908800FE06A48C08C6A490988884241
S113553009D16748008D67494988884203D1664983
S11355406648FFF7F5FE10BD10B56149C98B674A7F
S1135550128891420CD15E49098C644A5288914266
S113556006D1062262495A4C2000FFF769FB93E0FA
S11355705749C98B5F4A12881140564A12885D4BBD
S11355801B881A4091420BD15149098C594A5288BF
S11355901140504A5288574B5B881A40914208D0B8
S11355A055490988554A118053494988534A5180BD
S11355B007E04749C98B514A11804549098C4F4A34
S11355C0518000213C4A117004E03B490978491C90
S11355D0394A11703849097808290FDA37483649A9
S11355E009780C22514308444449098802889142AD
S11355F0EBD14249498842889142E6D12E49097843
S1135600082943D10621FF22314C200000F0E8FF95
S113561006210022324C200000F0E2FF062231492C
S1135620314C2000FFF70CFB06222E492A4C2000A7
S1135630FFF706FB314800882549C8842F48408875
S113564023490885234800882149888321484088C4
S11356501F49C8834FF480701D4988824FF48070BD
S11356601B49C88108201A490882062018498874F1
S113567004201749C8744FF4C16015498881204833
S1135680204908602A201149088013E00622011DE0
S11356900F4C2000FFF7D4FA06221249124C2000C6
S11356A0FFF7CEFA08200A498881084800880E309E
S11356B00649088010BD000095180020C01600207F
S11356C097180020981800209618002082180020AF
S11356D0080200205C1800201E0200202402002082
S11356E028020020381800200E020020987D0000B7
S11356F0847D000064180020601800207C180020BD
S11357003E0200206818002038B504000D00DFF8C0
S1135710F003844204D05D21DFF8E803FEF73CF88F
S11357206808DFF8E413B0FBF1F000F0FF0014F1B7
S11357302401086031BD38B504000D00DFF8C00352
S1135740844204D0A621DFF8BC03FEF725F8DFF875
S1135750BC03054204D0AA21DFF8A803FEF71CF815
S113576014F10C00006830F0160005F0FF01084346
S113577014F10C01086014F10800006830F00E0008
S1135780C5F30721084314F10801086014F13C0033
S1135790006840084000C5F30741084314F13C0188
S11357A0086031BD70B582B004000D006E46DFF8AC
S11357B05003844205D040F21311DFF84803FDF78B
S11357C0EBFF002D05D14FF48A71DFF83803FDF7A4
S11357D0E3FF2878307068787070A878B070E87843
S11357E0F070009814F114010860002000902879EA
S11357F0307068797070009814F11801086073BDF6
S113580010B50400DFF8F802844205D040F26911B3
S1135810DFF8F002FDF7C0FF14F10800006850F053
S1135820100014F10801086014F10800006850F039
S1135830010014F10801086014F10C00006850F034
S1135840010014F10C01086014F10800006850F024
S1135850100014F10801086010BDF0B4002410F128
S113586010031D68ABB22E0C0E55641C2D0E0D5585
S1135870641C9D1FAA4201DA160006E09E1F04E084
S113588010F110052D680D51241D351FA542F7DABE
S1135890B44224DA10F110052D68F71EBC4209D178
S11358A00D55641C2E0A0E55641C2D0C0D55641CDC
S11358B0641C14E0B71EBC4206D10D55641C2D0AAD
S11358C00D55641CA41C0AE0761EB44207D10D5584
S11358D0641CE41C03E010F110010D68241D991EE2
S11358E08C42F8DB9B1F9A4201DA584200E0180010
S11358F0F0BC704770B504000D001600DFF800021C
S1135900844205D040F28F21DFF8F801FDF744FF0F
S1135910002D05D14FF42471DFF8E801FDF73CFFB9
S1135920012E05DA40F29121DFF8D801FDF734FFAA
S113593014F13400006810F03F0F01D1002004E09E
S1135940320029002000FFF788FF70BD30B4030047
S11359501000002240F2FF74A04201DB404241E00B
S1135960B0F10E048D5C54EA0544521C8D5C54EA7B
S11359700564521C13F110052C6004E08C5813F1DB
S113598010052C60121D041F9442F7DA824225D0C0
S1135990C41EA2420DD18C5C521C8D5C54EA0524B9
S11359A0521C895C54EA0144521C13F110010C602E
S11359B014E0841EA24209D18C5C521C895C54EA16
S11359C00124521C13F110010C6007E0441EA24292
S11359D004D18C5C521C13F110010C60012113F1F1
S11359E03802116030BC704770B504000D00160019
S11359F04348844204D040F29E314248FDF7CCFE35
S1135A00002D04D140F29F313E48FDF7C5FE012E22
S1135A1004DA4FF468713B48FDF7BEFE14F1380018
S1135A200068C007FAD4320029002000FFF78EFF77
S1135A3070BD38B504000D003148844204D040F2F2
S1135A4047413048FDF7A8FEE809C001002804D00A
S1135A5040F24A412B48FDF79FFE201D0068A843F1
S1135A60211D086031BD38B504000D00244884426E
S1135A7004D040F26A412348FDF78EFE2068EDB25F
S1135A80002D02D0211D0968084032BD38B504003C
S1135A900D001B48844204D040F29F411948FDF791
S1135AA07BFEE809C001002804D040F2A241154859
S1135AB0FDF772FE256031BD38B504000D001048B5
S1135AC0844204D040F212510E48FDF765FE14F1F1
S1135AD020000068C007FAD4EDB2E80010F0F80026
S1135AE050F0010014F12001086014F12000006856
S1135AF0C007FAD414F13000006880B232BD00004F
S1135B000080044094760000A0252600E9F1FEFF01
S1135B1010B50400A00504D09C21DFF86001FDF756
S1135B203BFE40F60120DFF858110860DFF854010D
S1135B300460DFF85401DFF854110860DFF84C0109
S1135B4000688007FAD4DFF84801006840F60121B4
S1135B50084202D05FF0FF3000E0002010BD70B5B5
S1135B6004000D00160015F0030F04D0DF21DFF848
S1135B700C01FDF711FE16F0030F04D0E021DFF84D
S1135B80FC00FDF709FE42F20160DFF8F410086042
S1135B90DFF800010068C0073AD5002E3AD0E809C2
S1135BA0C001DFF8E010086009E0206815F07C010E
S1135BB0DFF8E42051180860241D2D1D361F15F050
S1135BC07C0F04D1DFF8D4000068002801D1002E36
S1135BD0EBD1DFF8CC00DFF8CC100860DFF8C400AC
S1135BE00068C007FAD4D8E7DFF898000560206899
S1135BF0DFF8B4100860DFF8A800DFF89010086040
S1135C00DFF888000068C007FAD4241D2D1D361F54
S1135C10002EE9D1DFF87800006842F20161084201
S1135C2002D05FF0FF3000E0002070BD38B5040002
S1135C300D00002C04D14FF421711048FDF7ACFD88
S1135C40002D04D140F285210C48FDF7A5FD17482D
S1135C50006810F0E04F06D014480068144908406A
S1135C60B0F1805F02D15FF0FF3006E011480068B8
S1135C702060114800682860002032BDF4760000DE
S1135C8014D00F4000D00F40020042A408D00F40AF
S1135C900CD00F40A0E10F4000D10F4030D00F4096
S1135CA0010042A420D00F4004D00F4000E00F4078
S1135CB00000FF70E0E10F40E4E10F4080B5FFF722
S1135CC0B9F800F0C1FC002031490870FEF798FED5
S1135CD003202F49087001BD80B52E4800F0EFFC69
S1135CE0012805D100202A4908702A48FFF7CCF87A
S1135CF02848FEF7F1FE012805D103202449087045
S1135D002448FFF7C1F801BD704738B504000D0001
S1135D101F480078002804D12900C9B2200000F0EF
S1135D20A1FC1B480078032804D12900C9B2200033
S1135D30FEF7AEFEFFF7A2F831BD15480078002843
S1135D4005D0022807D004D3032806D007E040205A
S1135D5006E0002004E0002002E0402000E04020B3
S1135D6080B270470A480078002805D0022807D07E
S1135D7004D3032806D007E0402006E0002004E016
S1135D80002002E0402000E0402080B27047000084
S1135D9000000020B017002080B5FFF766F802BDB0
S1135DA080B50020DFF86C160870DFF86C16002050
S1135DB0FBF7EDFBC0B2002804D07721DFF85C06C6
S1135DC0FDF7EAFC01BDDFF84C060078002801D19C
S1135DD0012000E00020704780B5FFF7DDFF0128B7
S1135DE001D1002011E0DFF82C060078002801D052
S1135DF000200AE000F0DAFC012805D10120DFF8D8
S1135E0014160870012000E0002002BD10B5002423
S1135E10DFF800060078002800F0FF81DFF8F405C1
S1135E200078012836D100F08AFB00F0D9FCDFF8B5
S1135E30F00500F00AFDDFF8EC0500F006FD00F0C7
S1135E40CDFC01220100DFF8E005FBF7B9FB0028D7
S1135E5007D0DFF8D80500F0F8FC012000F0EBFCD7
S1135E60DBE1DFF8CC0500F0F0FCDFF8C80500F05A
S1135E70ECFCDFF8C40500F0E8FC0020DFF8BC15FA
S1135E8008600020DFF8B41548600220DFF88415AC
S1135E900870C2E1DFF87C050078022840F0F68043
S1135EA0DFF884254FF48071DFF89405FCF70CF8D3
S1135EB0DFF8641591F83A12C9B2C909C9B20129C7
S1135EC00FDBDFF8680500F0C0FC022000F0B3FC33
S1135ED0DFF85405FBF781FE0020DFF83815087061
S1135EE09BE100281BD00022DFF85815DFF850058D
S1135EF000F0D4F9040024B214F1010F0FD1DFF83B
S1135F002C0500F0A2FC032000F095FCDFF8180536
S1135F10FBF763FE0020DFF8FC1408707DE124B277
S1135F20012C28DBDFF81405406800280BD1DFF8CA
S1135F301005D0F88001DFF80415086024B2DFF8FA
S1135F40FC04446017E0DFF8F804D0F88001DFF8BF
S1135F50EC140968884206D2DFF8E404D0F8800122
S1135F60DFF8D8140860DFF8D404406824B220189D
S1135F70DFF8C8144860DFF8A004D0F83C02DFF86A
S1135F809814D1F84012884201D1012000E0002089
S1135F900128C0F242810021DFF88C04FBF729FEBE
S1135FA000280FD0DFF8840400F04FFC042000F038
S1135FB042FCDFF87404FBF710FE0020DFF85414F1
S1135FC008702AE1DFF8680400F03FFCDFF8780489
S1135FD000F03BFCDFF87414DFF86004406800F064
S1135FE070FADFF8680400F030FCDFF8640400F0B5
S1135FF02CFCDFF85814DFF844040068000EC0B22B
S113600000F04DFADFF84C14DFF830040068000C9F
S1136010C0B200F044FADFF84014DFF8200400684E
S1136020000AC0B200F03BFADFF83014DFF80C04C9
S11360300068C0B200F033FADFF8100400F005FC89
S113604076A000F002FCDFF8F4034168DFF8EC030B
S1136050006800F07CFA00280FD1DFF8D00300F0CC
S1136060F4FB052000F0E7FBDFF8BC03FBF7B5FD0C
S11360700020DFF8A0130870CFE0DFF8B40300F0CD
S1136080E4FB0320DFF88C130870C6E0DFF8840318
S11360900078032840F0C180DFF88C234FF480712E
S11360A0DFF89C03FBF710FFDFF86C1391F83A124A
S11360B0C9B2C909C9B201290EDBDFF8A40300F093
S11360C0C4FB022000F0B7FBDFF85C03FBF785FD9F
S11360D00020D0490870A0E000281AD0DFF88423FB
S11360E0DFF86013DFF8580300F0D8F8040024B296
S11360F014F1010F0DD1DFF8700300F0A6FB0320AB
S113610000F099FBC848FBF768FD0020C1490870FE
S113611083E024B2012C4CDBD44800F096FBCB493D
S113612024B2200000F0CDF9C84800F08EFBD0481E
S113613000F08BFBC549C248D0F88001000EC0B204
S113614000F0ADF9C349BE48D0F88001000CC0B2DC
S113615000F0A5F9C049BA48D0F88001000AC0B2DD
S113616000F09DF9BD49B648D0F88001C0B200F0F6
S113617096F9B64800F069FB28A000F066FBB94A1E
S113618024B22100AE48D0F8800100F0DCF90028E8
S11361900CD1A64800F059FB062000F04CFBA248A5
S11361A0FBF71BFD00209B49087036E0A04800F077
S11361B04CFB9948D0F83C029749D1F840128842E8
S11361C001D1012000E00020012826DBA94800F0CD
S11361D03CFB00F0C8F900280CD1944800F035FBD2
S11361E0072000F028FB9048FBF7F7FC00208949C2
S11361F0087012E08E4800F028FB9F4800F025FB51
S11362008948FBF7EAFC9D4800F01FFB0020814908
S1136210087000F0F6FA00F0B5F910BD2E2E2E002D
S113622010B50400207800F03BFB532804D16078BB
S113623000F03CFB002801D103200FE060783128F6
S113624001D100200AE06078322801D1012005E064
S11362506078332801D1022000E0032010BD70B51E
S113626004000026A41C200000F044F90500AE1927
S1136270A41C200000F03EF986196D1EA41CADB2CA
S1136280022DF6DAF6B2F643200000F033F9F6B246
S1136290864201D0002000E0012070BD2DE9F041CC
S11362A007000C0015005FF00008002C01D0002F3F
S11362B004D140F233215948FDF76EFA3800FFF754
S11362C0AFFF0600F6B2032E01D10020A0E0380093
S11362D0FFF7C5FF002802D15FF0FF3098E0F6B267
S11362E0002E03D0022E58D027D38FE0BF1C3800D5
S11362F000F000F90600BF1C380000F0FBF80002B3
S11363002060BF1C380000F0F5F82168C0B24018C6
S11363102060BF1CB6F10308002D0DD0002406E058
S1136320380000F0E7F8A4B22855BF1C641CA4B2DE
S11363300FFA88F84445F3DB68E0BF1C380000F02E
S1136340D9F80600BF1C380000F0D4F8000420601F
S1136350BF1C380000F0CEF82168C0B211EB002059
S11363602060BF1C380000F0C5F82168C0B2401896
S11363702060BF1CB6F10408002D0DD0002406E0F7
S1136380380000F0B7F8A4B22855BF1C641CA4B2AE
S11363900FFA88F84445F3DB38E0BF1C380000F0FE
S11363A0A9F80600BF1C380000F0A4F8000620601D
S11363B0BF1C380000F09EF82168C0B211EB004009
S11363C02060BF1C380000F095F82168C0B211EBC2
S11363D000202060BF1C380000F08CF82168C0B297
S11363E040182060BF1CB6F10508002D0DD0002414
S11363F006E0380000F07EF8A4B22855BF1C641CE7
S1136400A4B20FFA88F84445F3DBFFE7404600B234
S1136410BDE8F0818F1800204C080020587A000055
S1136420607B0000107B0000800A0020747D000067
S11364307C7D0000847B0000887A000030180020F6
S1136440D4140020541600203C7D0000F0170020D6
S1136450147C0000F2170020F4170020F617002027
S1136460A87B0000D4150020CC7B0000007D000038
S1136470AC7C0000307C0000C47C0000B87A0000D2
S113648080B5010011F00F003030C9B20A2901DBD8
S1136490C01D02E0C0B200F003FAC0B202BD38B5BC
S11364A004000D002000C0B20009FFF7E9FF2870C6
S11364B014F00F00FFF7E4FF68700020A8702800B4
S11364C032BD0200491C0A23B2FBF3F2002AF9D1BF
S11364D000220A700200491E0A20B2FBF0F300FBFE
S11364E01320303008700A20B2FBF0F2002AF2D1F7
S11364F00800704770B504000025002609E0303814
S1136500C0B20A2800DBC01FEDB2C0B210EB051503
S1136510761CF6B2022E0FDAF6B2A05D00F0C0F9D6
S1136520C0B2B0F13001172904D2C0B2B0F13A01BF
S11365300729E4D2002001E02800C0B270BD80B574
S113654000F0BAF901BD80B500F0C1F902BD80B513
S113655000F0E7F902BD80B500F041FA02BD80B554
S113656000F087FA02BD80B500F0F5F9002801D1EA
S1136570002001E000F062FA02BD000080B500F0E6
S1136580CFFB01BD10B5FFF7E6FF002810D0FFF7E1
S1136590BBFBFDF7E4F8FFF7E2FF064908400649B4
S11365A00860FFF7DCFF001D046800F0BBFBA04798
S11365B010BD000080FFFF1F08ED00E070B504006F
S11365C00D00160005E0287820706D1C641CFDF792
S11365D0E8F83000461E80B20028F4D170BD0000F7
S11365E062F30F2262F31F42401810F0030308D035
S11365F0C91A1FD3DB0748BF00F8012D28BF20F8B4
S1136600022D130030B414461546103928BF20E972
S11366103C00FAD8490728BF20E90C0048BF40F8DD
S1136620042D890028BF20F8022D48BF00F8012D51
S113663030BC7047C91818BF00F8012DCB0728BF1C
S113664000F8012D7047000080B55048FCF7C3FDE9
S1136650FCF740FF60234FF4614201004C4800F016
S113666088FB01BD70B504000D00EDB2412D03DBC4
S11366705B214848FDF790F82800C0B200F072F89A
S1136680C0B2012803D05F214248FDF785F80026F7
S11366900DE0FDF786F8B6B2A05D00F063F8C0B275
S11366A0012803D068213B48FDF776F8761C3000BA
S11366B02900C9B280B289B28842EAD370BD10B54C
S11366C0040035480078002813D1344800F03DF820
S11366D0012838D131480078002834D0FDF74DF82E
S11366E02F49086000202F49087001202A490870AA
S11366F029E02A482B4909780844401C00F025F871
S1136700012816D127480078401C264908702548DE
S1136710007822490978884215D12248027892B239
S113672021492000FFF74AFF00201B49087001207F
S11367300AE0FDF722F81A4909686431814202D25D
S1136740002015490870002010BD10B50400104841
S113675000F0EDFB10F1010F02D02070012000E0E9
S1136760002010BD80B50100C9B2094800F0F6FB55
S1136770002803D1002007E0FDF713F8044800F0D7
S1136780BFFB0028F8D0012002BD0000010000106A
S113679000C00040B0790000911800206C17002060
S11367A058180020901800206D17002000B589B0FB
S11367B06846202100F01AFC69463548FBF7EAFADE
S11367C0002808D10098002805D09DF80800C006CC
S11367D001D4012000E0002009B000BD2C4870471E
S11367E080B500202B4981F824020A222A4929482D
S11367F0FAF7E6FE002803D10120264981F8240295
S113680001BD10B5234890F82402012802D1214883
S1136810FBF7E3F9FCF7B1FF10F164041F4800F043
S1136820B6FB012803D1FCF7A8FF8442F6D218482E
S1136830FBF7DAFA10BD80B5164890F82402012857
S113684002D11448FBF7C9F901BD10B50400114881
S113685090F82402012817D10E492000FBF777FB9A
S1136860002811D500200B4981F824020948FBF7C0
S1136870B4F909E02178094800F070FB074800F0FA
S11368803FFB0028FAD0641C20780028F2D110BD08
S11368904C7C0000A40C0020107D000000C00040CF
S11368A0A0F161011A2938BF2038704730380A280E
S11368B08041C00F704700005FF0FF30DFF85414D0
S11368C008605FF0FF30DFF850140860704770B55F
S11368D004000D001600200000F0B0F9FF2805D0D8
S11368E02819401E00F0AAF9FF2801D1002017E062
S11368F0600A4FF400714843DFF8201409688842A5
S113690007D12B0032002100DFF80C0400F0E6F878
S113691006E02B0032002100DFF8F80300F0DEF877
S113692070BD70B504000D00200000F087F906006A
S11369302819401E00F082F9F6B2FF2E02D0C0B230
S1136940FF2801D1002005E00100C9B23000C0B227
S113695000F031F970BD80B500200090DFF8B80375
S1136960006810F1010F01D1012037E00098DFF831
S1136970A8134968081800900098DFF89C138968E8
S1136980081800900098DFF89013C9680818009060
S11369900098DFF884130969081800900098DFF85C
S11369A078134969081800900098DFF86C13896916
S11369B0081800900098DFF86013C969081800905F
S11369C00098C04300900098401C00906A4604213F
S11369D0DFF848030068F030FFF779FF02BD0020BC
S11369E0DFF83813096809680818CC490968091DD3
S11369F009680818C9490968083109680818C749A5
S1136A0009680C3109680818C44909681031096813
S1136A100818C2490968143109680818BF49096887
S1136A20183109680818BD490968F031096808185F
S1136A30002801D1012000E00020704780B5B6484D
S1136A40006810F1010F06D0B34800F08AF800285E
S1136A5001D100200CE0AF48006810F1010F06D00E
S1136A60AC4800F07EF8002801D1002000E00120AD
S1136A7002BDAA480068704780B5CA0501D000204D
S1136A800BE002688A4201D1012006E001604FF464
S1136A900072001DFFF792FD012002BD38B504000D
S1136AA00D009D48844208D19A4C29002000FFF72C
S1136AB0E3FF002810D100200FE0984800688542C9
S1136AC003D1954C95480568EFE7200000F049F89C
S1136AD00028EAD1002000E0200032BD2DE9F04179
S1136AE004000F0015001E00780A4FF4007101FB2A
S1136AF000F8206810F1010F07D141462000FFF78C
S1136B00BBFF002801D1002029E02068404508D0BF
S1136B1041462000FFF7C2FF0400002C01D10020F1
S1136B201DE02068381A2044071DFCF73AFE201D9A
S1136B30381AB0F5007F0AD318F500712000FFF76A
S1136B40ADFF0400002C01D1002008E0271D2878A7
S1136B5038707F1C6D1C761E002EE6D10120BDE826
S1136B60F081F8B505000124286800F067F8C0B288
S1136B70FF2801D100201DE0002600E0761C802EB5
S1136B8016D2286810EB860705EB86004068009053
S1136B90FCF707FE042239006846FEF7E0FF0028F0
S1136BA001D0002404E0386800998842E6D000242B
S1136BB02000C0B2F2BD70B50C0021000200C9B2C1
S1136BC0D2B2914201D2002037E00100534A127A36
S1136BD0C9B2914206D3514991F8BC102200D2B2F5
S1136BE0914201D2002028E0C0B200F053F8050021
S1136BF02000C0B200F04EF806002000C0B200F041
S1136C0068F88019401E401B401C840A002600E0DE
S1136C10761C3000210080B289B288420CD2FCF785
S1136C20C0FDB6B24FF4806000FB0650FEF770FF63
S1136C300028EDD0002000E0012070BD38B504002C
S1136C40002500E06D1CEDB2102D21D2FCF7A9FD4A
S1136C503248EDB20C2101FB05F140588442F1D3D6
S1136C602E48EDB20C2101FB05F140582B49EDB241
S1136C700C2202FB05F21144496808188442E1D24F
S1136C802648EDB20C2101FB05F10844007A00E02E
S1136C90FF2032BD38B50500002400E0641CE4B2D6
S1136CA0102C13D2FCF77DFD1C48E4B20C2101FB2F
S1136CB004F10844007A2900C9B28842EED1174889
S1136CC0E4B20C2101FB04F1405801E05FF0FF3015
S1136CD032BD38B50500002400E0641CE4B2102C79
S1136CE014D2FCF75EFD0D48E4B20C2101FB04F163
S1136CF00844007A2900C9B28842EED10748E4B2B8
S1136D000C2101FB04F10844406800E0002032BD7E
S1136D1000000000CC0E0020D0100020E874000019
S1136D2072B6704762B67047DFF8881288421BD08B
S1136D30DFF88412884217D0DFF88012884213D01B
S1136D40DFF87C1288420FD0DFF8781288420BD02B
S1136D50DFF87412884207D0DFF87012884203D03B
S1136D60DFF86C12884201D1012000E00020C0B29B
S1136D707047F8B504000E0017001D002000FFF74F
S1136D80D3FF002805D14FF4B071DFF84802FCF7B7
S1136D9003FD002F05D140F26111DFF83802FCF742
S1136DA0FBFCDFF83402006810F0E04F27D0DFF876
S1136DB028020068DFF824120840B0F1805F1ED07A
S1136DC0DFF814020068DFF814120840DFF810122C
S1136DD0884205D1DFF80002006880B202280ED094
S1136DE0DFF8F4010068DFF8F4110840DFF8F4116B
S1136DF0884206D1DFF8E0010068000401D11020C8
S1136E0000E0082000FB07F0864205D24FF4B17180
S1136E10DFF8C001FCF7C0FC200000F04DF8B6EB31
S1136E20071F09D214F13000006850F0200014F15B
S1136E30300108607F0807E014F13000006830F08A
S1136E40200014F130010860F000B0FBF7F0401CA2
S1136E504008810914F12402116010F03F0014F17C
S1136E602801086014F12C000560002014F11801B9
S1136E700860200000F001F8F1BD10B50400200006
S1136E80FFF752FF002805D14FF4FB71DFF84401EE
S1136E90FCF782FC14F12C00006850F0100014F18F
S1136EA02C01086014F13000006840F201310843FD
S1136EB014F13001086010BD10B504002000FFF784
S1136EC033FF002805D140F21621DFF80801FCF752
S1136ED063FC14F1180000680007FAD414F12C00C4
S1136EE0006830F0100014F12C01086014F1300037
S1136EF00068DFF8F410084014F13001086010BD98
S1136F0010B504002000FFF70FFF002805D140F260
S1136F105541DFF8C000FCF73FFC14F1180000688D
S1136F20400910F0010090F00100C0B210BD10B58E
S1136F3004002000FFF7F8FE002805D140F2764156
S1136F40DFF89000FCF728FC14F118000068C00674
S1136F5001D4206801E05FF0FF3010BD38B50400B3
S1136F600D002000FFF7E0FE002805D140F2C941E2
S1136F70DFF86000FCF710FC14F1180000688006CC
S1136F8003D4EDB22560012000E0002032BD10B52D
S1136F9004002000FFF7C8FE002804D140F23B5152
S1136FA00C48FCF7F9FB14F118000068C00810F055
S1136FB0010010BD00C0004000D0004000E00040CF
S1136FC000F000400000014000100140002001409A
S1136FD000300140B477000000E00F400000FF7073
S1136FE00000011000000310FEFCFFFF002200F06F
S1136FF001B8000000B500BF13009646944610394E
S113700028BFA0E80C50FAD85FEA417C28BF0CC026
S113701048BF40F8042BC90728BF20F8022B48BFFB
S113702000F8012B00BD00006100620063006400F1
S1137030650066006700680069006A006B006C0008
S11370406D006E006F0070007100720073007400B8
S1137050750076007700780079007A00A100A2001C
S1137060A300A500AC00AF00E000E100E200E300F3
S1137070E400E500E600E700E800E900EA00EB00D0
S1137080EC00ED00EE00EF00F000F100F200F30080
S1137090F400F500F600F800F900FA00FB00FC002B
S11370A0FD00FE00FF0001010301050107010901C4
S11370B00B010D010F011101130115011701190134
S11370C01B011D011F0121012301250127012901A4
S11370D02B012D012F0131013301350137013A0113
S11370E03C013E01400142014401460148014B017B
S11370F04D014F01510153015501570159015B01E4
S11371005D015F01610163016501670169016B0153
S11371106D016F0171017301750177017A017C01C1
S11371207E019201B103B203B303B403B503B60302
S1137130B703B803B903BA03BB03BC03BD03BE035F
S1137140BF03C003C103C303C403C503C603C7030A
S1137150C803C903CA0330043104320433043404B9
S1137160350436043704380439043A043B043C0437
S11371703D043E043F0440044104420443044404E7
S1137180450446044704480449044A044B044C0497
S11371904D044E044F045104520453045404550442
S11371A056045704580459045A045B045C045E04EE
S11371B05F0470217121722173217421752176215C
S11371C07721782179217A217B217C217D217E21DF
S11371D07F2141FF42FF43FF44FF45FF46FF47FF36
S11371E048FF49FF4AFF4BFF4CFF4DFF4EFF4FFF47
S11371F050FF51FF52FF53FF54FF55FF56FF57FFF7
S113720058FF59FF5AFF0000410042004300440068
S1137210450046004700480049004A004B004C0026
S11372204D004E004F0050005100520053005400D6
S1137230550056005700580059005A002100E0FF3D
S1137240E1FFE5FFE2FFE3FFC000C100C200C300AD
S1137250C400C500C600C700C800C900CA00CB00EE
S1137260CC00CD00CE00CF00D000D100D200D3009E
S1137270D400D500D600D800D900DA00DB00DC0049
S1137280DD00DE00780100010201040106010801AD
S11372900A010C010E01100112011401160118015A
S11372A01A011C011E0120012201240126012801CA
S11372B02A012C012E013001320134013601390139
S11372C03B013D013F0141014301450147014A01A1
S11372D04C014E01500152015401560158015A010A
S11372E05C015E01600162016401660168016A017A
S11372F06C016E01700172017401760179017B01E8
S11373007D019101910392039303940395039603E2
S11373109703980399039A039B039C039D039E037D
S11373209F03A003A103A303A403A503A603A70328
S1137330A803A903AA0310041104120413041404D7
S1137340150416041704180419041A041B041C0455
S11373501D041E041F042004210422042304240405
S1137360250426042704280429042A042B042C04B5
S11373702D042E042F040104020403040404050450
S113738006040704080409040A040B040C040E048C
S11373900F0460216121622163216421652166213A
S11373A06721682169216A216B216C216D216E217D
S11373B06F2121FF22FF23FF24FF25FF26FF27FF44
S11373C028FF29FF2AFF2BFF2CFF2DFF2EFF2FFF65
S11373D030FF31FF32FF33FF34FF35FF36FF37FF15
S11373E038FF39FF3AFF0000C700FC00E900E20063
S11373F0E400E000E500E700EA00EB00E800EF004D
S1137400EE00EC00C400C500C900E600C600F400AC
S1137410F600F200FB00F900FF00D600DC00A20039
S1137420A300A500A7209201E100ED00F300FA00FB
S1137430F100D100AA00BA00BF001023AC00BD00C7
S1137440BC00A100AB00BB00912592259325022529
S11374502425612562255625552563255125572563
S11374605D255C255B251025142534252C251C253C
S113747000253C255E255F255A255425692566256A
S1137480602550256C2567256825642565255925C3
S11374905825522553256B256A2518250C25882542
S11374A084258C2590258025B103DF009303C00338
S11374B0A303C303B500C403A6039803A903B40339
S11374C01E22C603B50329226122B100652264226B
S11374D020232123F7004822B0001922B7001A22E2
S11374E07F20B200A025A000008000000020000042
S11374F00400000000A000000020000005000000BF
S113750000C00000002000000600000000E00000B1
S1137510002000000700000000000100002000001F
S11375200800000000200100002000000900000005
S113753000400100002000000A000000006001007B
S1137540002000000B00000000800100002000006B
S11375500C00000000A00100002000000D0000004D
S113756000C00100002000000E00000000E0010047
S1137570002000000F000000000002000080000056
S113758010000000008002000080000011000000D4
S113759000000300008000001200000000800300CF
S11375A00080000013000000809A90418E418F807B
S11375B04545454949498E8F9092924F994F55556B
S11375C059999A9B9C9D9E9F41494F55A5A5A6A755
S11375D0A8A9AAABAC21AEAFB0B1B2B3B4B5B6B73B
S11375E0B8B9BABBBCBDBEBFC0C1C2C3C4C5C6C79F
S11375F0C8C9CACBCCCDCECFD0D1D2D3D4D5D6D78F
S1137600D8D9DADBDCDDDEDFE0E1E2E3E4E5E6E77E
S1137610E8E9EAEBECEDEEEFF0F1F2F3F4F5F6F76E
S1137620F8F9FAFBFCFDFEFF40420F0000201C00AD
S113763080841E0000802500999E3600004038009A
S113764000093D0000803E0000004B00404B4C0010
S113765000204E00808D5B0000C05D000080700043
S113766000127A0000007D0080969800001BB7008D
S11376700080BB00C0E8CE00647ADA000024F40085
S11376800000FA0080A81201002D310100366E01BD
S113769040787D01433A5C576F726B5C736F66741C
S11376A0776172655C4F70656E424C545C546172D4
S11376B06765745C44656D6F5C41524D434D335F47
S11376C04C4D33535F454B5F4C4D33533639363550
S11376D05F4941525C426F6F745C6C69625C6472B6
S11376E0697665726C69625C65746865726E6574EE
S11376F02E630000433A5C576F726B5C736F667461
S1137700776172655C4F70656E424C545C54617273
S11377106765745C44656D6F5C41524D434D335FE6
S11377204C4D33535F454B5F4C4D335336393635EF
S11377305F4941525C426F6F745C6C69625C647255
S1137740697665726C69625C666C6173686C6962A7
S11377502E630000433A5C576F726B5C736F667400
S1137760776172655C4F70656E424C545C54617213
S11377706765745C44656D6F5C41524D434D335F86
S11377804C4D33535F454B5F4C4D3353363936358F
S11377905F4941525C426F6F745C6C69625C6472F5
S11377A0697665726C69625C73797363746C2E6359
S11377B000000000433A5C576F726B5C736F667431
S11377C0776172655C4F70656E424C545C546172B3
S11377D06765745C44656D6F5C41524D434D335F26
S11377E04C4D33535F454B5F4C4D3353363936352F
S11377F05F4941525C426F6F745C6C69625C647295
S1137800697665726C69625C756172746C69622E0A
S11378106300000080B5012014490870FBF7ADFF38
S11378201349086000F001F801BD80B5FEF7B4FA11
S1137830012819D0FEF7C7FA002815D00B480078A4
S1137840012811D1FBF799FF0949096801F51C5179
S11378501031884208D3002004490870FEF7BCFAAE
S1137860002801D1FEF78EFE01BD00008E18002015
S113787040180020433A5C576F726B5C736F6674F8
S1137880776172655C4F70656E424C545C546172F2
S11378906765745C44656D6F5C41524D434D335F65
S11378A04C4D33535F454B5F4C4D3353363936356E
S11378B05F4941525C426F6F745C6C69625C6472D4
S11378C0697665726C69625C6770696F2E6300002B
S11378D0433A5C576F726B5C736F66747761726561
S11378E05C4F70656E424C545C5461726765745CA5
S11378F044656D6F5C41524D434D335F4C4D335382
S11379005F454B5F4C4D3353363936355F494152F1
S11379105C426F6F745C6C69625C647269766572F8
S11379206C69625C7373692E63000000433A5C57B0
S11379306F726B5C736F6674776172655C4F7065B0
S11379406E424C545C5461726765745C536F75721B
S113795063655C41524D434D335F4C4D33535C4939
S113796041525C766563746F72732E63000000008D
S113797019E050F8041BCB0744BFA9F101035918BF
S1137980121F0023042A41F8043BF9D25FEA827CE7
S11379900B4604D54FF0000CA1F800C09B1CD10786
S11379A044BF0021197050F8042B002AE1D170471C
S11379B0433A5C576F726B5C736F66747761726580
S11379C05C4F70656E424C545C5461726765745CC4
S11379D0536F757263655C41524D434D335F4C4D3B
S11379E033535C756172742E6300000080B5FEF73A
S11379F0C5FDFBF7D5FEFBF7A1FEFEF7A0FDFEF7E4
S1137A00CFF9FEF75BF9FFF705FF01BD80B5FBF782
S1137A10C8FEFBF7A8FEFEF7F9F9FEF75DF9FFF7DC
S1137A2004FF01BD80B500F005F8FFF7DFFFFFF7A5
S1137A30EDFFFCE780B50648FBF74CFC0548FBF777
S1137A40CAFB03215FF04020FBF7E8F801BD00000A
S1137A508003C00101000020433A5C576F726B5CE5
S1137A60736F6674776172655C4F70656E424C54D7
S1137A705C5461726765745C536F757263655C66B0
S1137A80696C652E6300000050617273696E672033
S1137A906669726D776172652066696C6520746FC2
S1137AA0206F627461696E20657261736520736909
S1137AB07A652E2E2E0000004669726D776172651C
S1137AC02075706461746520737563636573736690
S1137AD0756C6C7920636F6D706C657465640A0DE8
S1137AE00000000010B450F8041B79B10268436828
S1137AF002440830DC0744BFA9F10104E31852F83A
S1137B00044B43F8044B091FF9D1ECE710BC704750
S1137B104F70656E696E67206669726D7761726514
S1137B202066696C6520666F722072656164696E97
S1137B30672E2E2E0000000010B507497944183135
S1137B40064C7C44163404E00A68081D1144884736
S1137B500146A142F8D110BD98000000B800000011
S1137B604669726D77617265207570646174652011
S1137B707265717565737420646574656374656496
S1137B800A0D00005374617274696E67207468652D
S1137B902070726F6772616D6D696E6720736571B5
S1137BA075656E63650A0D0052656164696E6720D0
S1137BB06C696E652066726F6D2066696C652E2E29
S1137BC02E4552524F520A0D00000000496E766154
S1137BD06C696420636865636B73756D20666F758B
S1137BE06E642E2E2E4552524F520A0D0000000094
S1137BF081FDFFFF94160000080200200000000031
S1137C00E5FEFFFF040000009401000000000020D6
S1137C10000000002062797465732066726F6D2025
S1137C206D656D6F727920617420307800000000FA
S1137C3057726974696E672070726F6772616D2024
S1137C40636865636B73756D2E2E2E002F64656DEE
S1137C506F70726F675F656B5F6C6D337336393647
S1137C60352E73726563000000F00BF8002801D014
S1137C70FFF762FF0020AFF30080FFF7D3FE00F0B0
S1137C8002F80120704700F001B8000007463846AA
S1137C9000F002F8FBE7000080B5AFF30080024A71
S1137CA011001820ABBEFBE72600020020627974A5
S1137CB0657320746F206D656D6F72792061742017
S1137CC030780000436C6F73696E67206669726D6B
S1137CD0776172652066696C650A0D00034B9D46E9
S1137CE0AFF30080AFF30080FFF7BEFF080200206F
S1137CF001030507090E10121416181C1E000000BB
S1137D0050726F6772616D6D696E672000000000CC
S1137D102F626F6F746C6F672E74787400000000AC
S1137D2080B53C210148FBF737FD01BD2C790000EB
S1137D30222A3A3C3E3F7C7F00000000457261737A
S1137D40696E67200000000040E00F4044E00F40EF
S1137D5048E00F4000E10F4004E10F4008E10F400C
S1137D60AFF30080AFF30080FFF77EFF2B2C3B3D89
S1137D705B5D00004552524F520A0D004F4B0A0DF5
S1137D8000000000FFFFFFFFFFFF00004F70656E63
S1137D90424C540000000000FFFFFFFF04010000FC
S9037D611E
